 nio

 Timestamp is eade0304 (reproducible build file hash)

 Preferred load address is 0000000180000000

 Start         Length     Name                   Class
 0001:00000000 00006f40H .text$mn                CODE
 0001:00006f40 00000036H .text$mn$00             CODE
 0001:00006f76 00000092H .text$x                 CODE
 0002:00000000 00000560H .idata$5                DATA
 0002:00000560 00000038H .00cfg                  DATA
 0002:00000598 00000008H .CRT$XCA                DATA
 0002:000005a0 00000008H .CRT$XCZ                DATA
 0002:000005a8 00000008H .CRT$XIA                DATA
 0002:000005b0 00000008H .CRT$XIZ                DATA
 0002:000005b8 00000008H .CRT$XPA                DATA
 0002:000005c0 00000008H .CRT$XPZ                DATA
 0002:000005c8 00000008H .CRT$XTA                DATA
 0002:000005d0 00000010H .CRT$XTZ                DATA
 0002:000005d8 00000000H .gehcont$y              DATA
 0002:000005d8 00000000H .gfids$y                DATA
 0002:000005e0 00000aa0H .rdata                  DATA
 0002:00001080 00000000H .rdata$CastGuardVftablesA DATA
 0002:00001080 00000000H .rdata$CastGuardVftablesC DATA
 0002:00001080 0000006cH .rdata$voltmd           DATA
 0002:000010ec 000002b4H .rdata$zzzdbg           DATA
 0002:000013a0 00000008H .rtc$IAA                DATA
 0002:000013a8 00000008H .rtc$IZZ                DATA
 0002:000013b0 00000008H .rtc$TAA                DATA
 0002:000013b8 00000008H .rtc$TZZ                DATA
 0002:000013c0 00000700H .xdata                  DATA
 0002:00001ac0 00002880H .edata                  DATA
 0002:00004340 000000dcH .idata$2                DATA
 0002:0000441c 00000014H .idata$3                DATA
 0002:00004430 00000560H .idata$4                DATA
 0002:00004990 00000c30H .idata$6                DATA
 0003:00000000 00000050H .data                   DATA
 0003:00000050 00000748H .bss                    DATA
 0004:00000000 00000924H .pdata                  DATA
 0005:00000000 00000060H .rsrc$01                DATA
 0005:00000060 00000300H .rsrc$02                DATA

  Address         Publics by Value              Rva+Base               Lib:Object

 0000:00000000       __AbsoluteZero             0000000000000000     <absolute>
 0000:00000000       ___safe_se_handler_count   0000000000000000     <absolute>
 0000:00000000       ___safe_se_handler_table   0000000000000000     <absolute>
 0000:00000000       __arm64x_extra_rfe_table   0000000000000000     <absolute>
 0000:00000000       __arm64x_extra_rfe_table_size 0000000000000000     <absolute>
 0000:00000000       __arm64x_native_entrypoint 0000000000000000     <absolute>
 0000:00000000       __arm64x_redirection_metadata 0000000000000000     <absolute>
 0000:00000000       __arm64x_redirection_metadata_count 0000000000000000     <absolute>
 0000:00000000       __dynamic_value_reloc_table 0000000000000000     <absolute>
 0000:00000000       __enclave_config           0000000000000000     <absolute>
 0000:00000000       __guard_check_icall_a64n_fptr 0000000000000000     <absolute>
 0000:00000000       __guard_eh_cont_count      0000000000000000     <absolute>
 0000:00000000       __guard_eh_cont_table      0000000000000000     <absolute>
 0000:00000000       __guard_fids_count         0000000000000000     <absolute>
 0000:00000000       __guard_fids_table         0000000000000000     <absolute>
 0000:00000000       __guard_iat_count          0000000000000000     <absolute>
 0000:00000000       __guard_iat_table          0000000000000000     <absolute>
 0000:00000000       __guard_longjmp_count      0000000000000000     <absolute>
 0000:00000000       __guard_longjmp_table      0000000000000000     <absolute>
 0000:00000000       __hybrid_auxiliary_delayload_iat 0000000000000000     <absolute>
 0000:00000000       __hybrid_auxiliary_delayload_iat_copy 0000000000000000     <absolute>
 0000:00000000       __hybrid_auxiliary_iat     0000000000000000     <absolute>
 0000:00000000       __hybrid_auxiliary_iat_copy 0000000000000000     <absolute>
 0000:00000000       __hybrid_code_map          0000000000000000     <absolute>
 0000:00000000       __hybrid_code_map_count    0000000000000000     <absolute>
 0000:00000000       __hybrid_image_info_bitfield 0000000000000000     <absolute>
 0000:00000000       __x64_code_ranges_to_entry_points 0000000000000000     <absolute>
 0000:00000000       __x64_code_ranges_to_entry_points_count 0000000000000000     <absolute>
 0000:00000100       __guard_flags              0000000000000100     <absolute>
 0000:00000000       __ImageBase                0000000180000000     <linker-defined>
 0001:00000000       Java_sun_nio_ch_DatagramChannelImpl_disconnect0 0000000180001000 f   DatagramChannelImpl.obj
 0001:000000c4       Java_sun_nio_ch_DatagramChannelImpl_initIDs 00000001800010c4 f   DatagramChannelImpl.obj
 0001:000001dc       Java_sun_nio_ch_DatagramChannelImpl_receive0 00000001800011dc f   DatagramChannelImpl.obj
 0001:000003cc       Java_sun_nio_ch_DatagramChannelImpl_send0 00000001800013cc f   DatagramChannelImpl.obj
 0001:000004a8       purgeOutstandingICMP       00000001800014a8 f   DatagramChannelImpl.obj
 0001:000005bc       Java_sun_nio_ch_DatagramDispatcher_read0 00000001800015bc f   DatagramDispatcher.obj
 0001:000006b4       Java_sun_nio_ch_DatagramDispatcher_readv0 00000001800016b4 f   DatagramDispatcher.obj
 0001:0000080c       Java_sun_nio_ch_DatagramDispatcher_write0 000000018000180c f   DatagramDispatcher.obj
 0001:000008f0       Java_sun_nio_ch_DatagramDispatcher_writev0 00000001800018f0 f   DatagramDispatcher.obj
 0001:00000a30       Java_sun_nio_ch_FileChannelImpl_initIDs 0000000180001a30 f   FileChannelImpl.obj
 0001:00000a8c       Java_sun_nio_ch_FileChannelImpl_map0 0000000180001a8c f   FileChannelImpl.obj
 0001:00000bb4       Java_sun_nio_ch_FileChannelImpl_transferTo0 0000000180001bb4 f   FileChannelImpl.obj
 0001:00000cac       Java_sun_nio_ch_FileChannelImpl_unmap0 0000000180001cac f   FileChannelImpl.obj
 0001:00000ce0       Java_sun_nio_ch_FileDispatcherImpl_close0 0000000180001ce0 f   FileDispatcherImpl.obj
 0001:00000d1c       Java_sun_nio_ch_FileDispatcherImpl_duplicateHandle 0000000180001d1c f   FileDispatcherImpl.obj
 0001:00000d7c       Java_sun_nio_ch_FileDispatcherImpl_force0 0000000180001d7c f   FileDispatcherImpl.obj
 0001:00000dcc       Java_sun_nio_ch_FileDispatcherImpl_lock0 0000000180001dcc f   FileDispatcherImpl.obj
 0001:00000eb4       Java_sun_nio_ch_FileDispatcherImpl_pread0 0000000180001eb4 f   FileDispatcherImpl.obj
 0001:00000fd4       Java_sun_nio_ch_FileDispatcherImpl_pwrite0 0000000180001fd4 f   FileDispatcherImpl.obj
 0001:000010c4       Java_sun_nio_ch_FileDispatcherImpl_read0 00000001800020c4 f   FileDispatcherImpl.obj
 0001:00001160       Java_sun_nio_ch_FileDispatcherImpl_readv0 0000000180002160 f   FileDispatcherImpl.obj
 0001:0000124c       Java_sun_nio_ch_FileDispatcherImpl_release0 000000018000224c f   FileDispatcherImpl.obj
 0001:00001300       Java_sun_nio_ch_FileDispatcherImpl_seek0 0000000180002300 f   FileDispatcherImpl.obj
 0001:00001368       Java_sun_nio_ch_FileDispatcherImpl_setDirect0 0000000180002368 f   FileDispatcherImpl.obj
 0001:000013fc       Java_sun_nio_ch_FileDispatcherImpl_size0 00000001800023fc f   FileDispatcherImpl.obj
 0001:00001444       Java_sun_nio_ch_FileDispatcherImpl_truncate0 0000000180002444 f   FileDispatcherImpl.obj
 0001:000014a0       Java_sun_nio_ch_FileDispatcherImpl_write0 00000001800024a0 f   FileDispatcherImpl.obj
 0001:00001550       Java_sun_nio_ch_FileDispatcherImpl_writev0 0000000180002550 f   FileDispatcherImpl.obj
 0001:0000164c       Java_sun_nio_ch_FileKey_init 000000018000264c f   FileKey.obj
 0001:00001700       Java_sun_nio_ch_FileKey_initIDs 0000000180002700 f   FileKey.obj
 0001:0000178c       Java_sun_nio_ch_IOUtil_configureBlocking 000000018000278c f   IOUtil.obj
 0001:00001810       Java_sun_nio_ch_IOUtil_drain 0000000180002810 f   IOUtil.obj
 0001:000018d8       Java_sun_nio_ch_IOUtil_fdVal 00000001800028d8 f   IOUtil.obj
 0001:000018ec       Java_sun_nio_ch_IOUtil_initIDs 00000001800028ec f   IOUtil.obj
 0001:00001968       Java_sun_nio_ch_IOUtil_iovMax 0000000180002968 f   IOUtil.obj
 0001:00001968       Java_sun_nio_ch_Net_polloutValue 0000000180002968 f   Net.obj
 0001:00001970       Java_sun_nio_ch_IOUtil_randomBytes 0000000180002970 f   IOUtil.obj
 0001:00001978       Java_sun_nio_ch_IOUtil_setfdVal 0000000180002978 f   IOUtil.obj
 0001:0000198c       convertLongReturnVal       000000018000298c f   IOUtil.obj
 0001:000019bc       convertReturnVal           00000001800029bc f   IOUtil.obj
 0001:000019e8       fdval                      00000001800029e8 f   IOUtil.obj
 0001:000019fc       handleval                  00000001800029fc f   IOUtil.obj
 0001:00001a10       Java_sun_nio_ch_Iocp_close0 0000000180002a10 f   Iocp.obj
 0001:00001a10       Java_sun_nio_fs_WindowsNativeDispatcher_CloseHandle 0000000180002a10 f   WindowsNativeDispatcher.obj
 0001:00001a1c       Java_sun_nio_ch_Iocp_createIoCompletionPort 0000000180002a1c f   Iocp.obj
 0001:00001a68       Java_sun_nio_ch_Iocp_getErrorMessage 0000000180002a68 f   Iocp.obj
 0001:00001a68       Java_sun_nio_fs_WindowsNativeDispatcher_FormatMessage 0000000180002a68 f   WindowsNativeDispatcher.obj
 0001:00001afc       Java_sun_nio_ch_Iocp_getQueuedCompletionStatus 0000000180002afc f   Iocp.obj
 0001:00001bc8       Java_sun_nio_ch_Iocp_initIDs 0000000180002bc8 f   Iocp.obj
 0001:00001c9c       Java_sun_nio_ch_Iocp_postQueuedCompletionStatus 0000000180002c9c f   Iocp.obj
 0001:00001cd4       Java_java_nio_MappedByteBuffer_force0 0000000180002cd4 f   MappedByteBuffer.obj
 0001:00001dc0       Java_java_nio_MappedByteBuffer_isLoaded0 0000000180002dc0 f   MappedByteBuffer.obj
 0001:00001dc0       Java_sun_nio_ch_Net_canIPv6SocketJoinIPv4Group0 0000000180002dc0 f   Net.obj
 0001:00001dc0       Java_sun_nio_ch_Net_canJoin6WithIPv4Group0 0000000180002dc0 f   Net.obj
 0001:00001dc0       Java_sun_nio_ch_Net_isReusePortAvailable0 0000000180002dc0 f   Net.obj
 0001:00001dc4       Java_java_nio_MappedByteBuffer_load0 0000000180002dc4 f   MappedByteBuffer.obj
 0001:00001dc4       _guard_check_icall_nop     0000000180002dc4 f   MSVCRT:guard_support.obj
 0001:00001dc8       Java_sun_nio_ch_Net_bind0  0000000180002dc8 f   Net.obj
 0001:00001e70       Java_sun_nio_ch_Net_blockOrUnblock4 0000000180002e70 f   Net.obj
 0001:00001f40       Java_sun_nio_ch_Net_blockOrUnblock6 0000000180002f40 f   Net.obj
 0001:00001f90       Java_sun_nio_ch_Net_connect0 0000000180002f90 f   Net.obj
 0001:00002198       Java_sun_nio_ch_Net_getIntOption0 0000000180003198 f   Net.obj
 0001:000022ac       Java_sun_nio_ch_Net_getInterface4 00000001800032ac f   Net.obj
 0001:00002310       Java_sun_nio_ch_Net_getInterface6 0000000180003310 f   Net.obj
 0001:00002370       Java_sun_nio_ch_Net_initIDs 0000000180003370 f   Net.obj
 0001:00002378       Java_sun_nio_ch_Net_isExclusiveBindAvailable 0000000180003378 f   Net.obj
 0001:00002378       Java_sun_nio_ch_Net_pollerrValue 0000000180003378 f   Net.obj
 0001:00002378       _get_startup_argv_mode     0000000180003378 f   MSVCRT:argv_mode.obj
 0001:00002380       Java_sun_nio_ch_Net_isIPv6Available0 0000000180003380 f   Net.obj
 0001:00002394       Java_sun_nio_ch_Net_joinOrDrop4 0000000180003394 f   Net.obj
 0001:000024a8       Java_sun_nio_ch_Net_joinOrDrop6 00000001800034a8 f   Net.obj
 0001:0000258c       Java_sun_nio_ch_Net_listen 000000018000358c f   Net.obj
 0001:0000258c       Java_sun_nio_ch_ServerSocketChannelImpl_listen 000000018000358c f   ServerSocketChannelImpl.obj
 0001:000025d8       Java_sun_nio_ch_Net_localInetAddress 00000001800035d8 f   Net.obj
 0001:00002658       Java_sun_nio_ch_Net_localPort 0000000180003658 f   Net.obj
 0001:000026e0       Java_sun_nio_ch_Net_poll   00000001800036e0 f   Net.obj
 0001:0000284c       Java_sun_nio_ch_Net_pollconnValue 000000018000384c f   Net.obj
 0001:00002854       Java_sun_nio_ch_Net_pollhupValue 0000000180003854 f   Net.obj
 0001:0000285c       Java_sun_nio_ch_Net_pollinValue 000000018000385c f   Net.obj
 0001:00002864       Java_sun_nio_ch_Net_pollnvalValue 0000000180003864 f   Net.obj
 0001:0000286c       Java_sun_nio_ch_Net_remoteInetAddress 000000018000386c f   Net.obj
 0001:000028ec       Java_sun_nio_ch_Net_remotePort 00000001800038ec f   Net.obj
 0001:00002974       Java_sun_nio_ch_Net_setIntOption0 0000000180003974 f   Net.obj
 0001:00002a4c       Java_sun_nio_ch_Net_setInterface4 0000000180003a4c f   Net.obj
 0001:00002ab0       Java_sun_nio_ch_Net_setInterface6 0000000180003ab0 f   Net.obj
 0001:00002b00       Java_sun_nio_ch_Net_shutdown 0000000180003b00 f   Net.obj
 0001:00002b5c       Java_sun_nio_ch_Net_socket0 0000000180003b5c f   Net.obj
 0001:00002d80       Java_sun_nio_fs_RegistryFileTypeDetector_queryStringValue 0000000180003d80 f   RegistryFileTypeDetector.obj
 0001:00002e58       Java_sun_nio_ch_ServerSocketChannelImpl_accept0 0000000180003e58 f   ServerSocketChannelImpl.obj
 0001:00002fa0       Java_sun_nio_ch_ServerSocketChannelImpl_initIDs 0000000180003fa0 f   ServerSocketChannelImpl.obj
 0001:0000305c       Java_sun_nio_ch_SocketChannelImpl_checkConnect 000000018000405c f   SocketChannelImpl.obj
 0001:000031cc       Java_sun_nio_ch_SocketChannelImpl_initIDs 00000001800041cc f   SocketChannelImpl.obj
 0001:00003214       Java_sun_nio_ch_SocketChannelImpl_sendOutOfBandData 0000000180004214 f   SocketChannelImpl.obj
 0001:00003264       handleSocketError          0000000180004264 f   SocketChannelImpl.obj
 0001:0000327c       Java_sun_nio_ch_SocketDispatcher_close0 000000018000427c f   SocketDispatcher.obj
 0001:000032b0       Java_sun_nio_ch_SocketDispatcher_preClose0 00000001800042b0 f   SocketDispatcher.obj
 0001:0000330c       Java_sun_nio_ch_SocketDispatcher_read0 000000018000430c f   SocketDispatcher.obj
 0001:000033cc       Java_sun_nio_ch_SocketDispatcher_readv0 00000001800043cc f   SocketDispatcher.obj
 0001:0000350c       Java_sun_nio_ch_SocketDispatcher_write0 000000018000450c f   SocketDispatcher.obj
 0001:000035e4       Java_sun_nio_ch_SocketDispatcher_writev0 00000001800045e4 f   SocketDispatcher.obj
 0001:00003768       Java_sun_nio_ch_WindowsAsynchronousFileChannelImpl_lockFile 0000000180004768 f   WindowsAsynchronousFileChannelImpl.obj
 0001:000037f8       Java_sun_nio_ch_WindowsAsynchronousFileChannelImpl_readFile 00000001800047f8 f   WindowsAsynchronousFileChannelImpl.obj
 0001:00003878       Java_sun_nio_ch_WindowsAsynchronousFileChannelImpl_writeFile 0000000180004878 f   WindowsAsynchronousFileChannelImpl.obj
 0001:000038ec       Java_sun_nio_ch_WindowsAsynchronousServerSocketChannelImpl_accept0 00000001800048ec f   WindowsAsynchronousServerSocketChannelImpl.obj
 0001:00003998       Java_sun_nio_ch_WindowsAsynchronousServerSocketChannelImpl_closesocket0 0000000180004998 f   WindowsAsynchronousServerSocketChannelImpl.obj
 0001:00003998       Java_sun_nio_ch_WindowsAsynchronousSocketChannelImpl_closesocket0 0000000180004998 f   WindowsAsynchronousSocketChannelImpl.obj
 0001:000039c4       Java_sun_nio_ch_WindowsAsynchronousServerSocketChannelImpl_initIDs 00000001800049c4 f   WindowsAsynchronousServerSocketChannelImpl.obj
 0001:00003aa8       Java_sun_nio_ch_WindowsAsynchronousServerSocketChannelImpl_updateAcceptContext 0000000180004aa8 f   WindowsAsynchronousServerSocketChannelImpl.obj
 0001:00003ad8       Java_sun_nio_ch_WindowsAsynchronousSocketChannelImpl_connect0 0000000180004ad8 f   WindowsAsynchronousSocketChannelImpl.obj
 0001:00003ba8       Java_sun_nio_ch_WindowsAsynchronousSocketChannelImpl_initIDs 0000000180004ba8 f   WindowsAsynchronousSocketChannelImpl.obj
 0001:00003c8c       Java_sun_nio_ch_WindowsAsynchronousSocketChannelImpl_read0 0000000180004c8c f   WindowsAsynchronousSocketChannelImpl.obj
 0001:00003d38       Java_sun_nio_ch_WindowsAsynchronousSocketChannelImpl_shutdown0 0000000180004d38 f   WindowsAsynchronousSocketChannelImpl.obj
 0001:00003d68       Java_sun_nio_ch_WindowsAsynchronousSocketChannelImpl_updateConnectContext 0000000180004d68 f   WindowsAsynchronousSocketChannelImpl.obj
 0001:00003d90       Java_sun_nio_ch_WindowsAsynchronousSocketChannelImpl_write0 0000000180004d90 f   WindowsAsynchronousSocketChannelImpl.obj
 0001:00003e34       Java_sun_nio_fs_WindowsNativeDispatcher_AccessCheck 0000000180004e34 f   WindowsNativeDispatcher.obj
 0001:00003f14       Java_sun_nio_fs_WindowsNativeDispatcher_AddAccessAllowedAceEx 0000000180004f14 f   WindowsNativeDispatcher.obj
 0001:00003f60       Java_sun_nio_fs_WindowsNativeDispatcher_AddAccessDeniedAceEx 0000000180004f60 f   WindowsNativeDispatcher.obj
 0001:00003fac       Java_sun_nio_fs_WindowsNativeDispatcher_AdjustTokenPrivileges 0000000180004fac f   WindowsNativeDispatcher.obj
 0001:00004028       Java_sun_nio_fs_WindowsNativeDispatcher_CancelIo 0000000180005028 f   WindowsNativeDispatcher.obj
 0001:00004054       Java_sun_nio_fs_WindowsNativeDispatcher_ConvertSidToStringSid 0000000180005054 f   WindowsNativeDispatcher.obj
 0001:000040c4       Java_sun_nio_fs_WindowsNativeDispatcher_ConvertStringSidToSid0 00000001800050c4 f   WindowsNativeDispatcher.obj
 0001:000040fc       Java_sun_nio_fs_WindowsNativeDispatcher_CopyFileEx0 00000001800050fc f   WindowsNativeDispatcher.obj
 0001:00004148       Java_sun_nio_fs_WindowsNativeDispatcher_CreateDirectory0 0000000180005148 f   WindowsNativeDispatcher.obj
 0001:00004194       Java_sun_nio_fs_WindowsNativeDispatcher_CreateEvent 0000000180005194 f   WindowsNativeDispatcher.obj
 0001:000041dc       Java_sun_nio_fs_WindowsNativeDispatcher_CreateFile0 00000001800051dc f   WindowsNativeDispatcher.obj
 0001:00004270       Java_sun_nio_fs_WindowsNativeDispatcher_CreateHardLink0 0000000180005270 f   WindowsNativeDispatcher.obj
 0001:000042a8       Java_sun_nio_fs_WindowsNativeDispatcher_CreateIoCompletionPort 00000001800052a8 f   WindowsNativeDispatcher.obj
 0001:000042f4       Java_sun_nio_fs_WindowsNativeDispatcher_CreateSymbolicLink0 00000001800052f4 f   WindowsNativeDispatcher.obj
 0001:0000432c       Java_sun_nio_fs_WindowsNativeDispatcher_DeleteFile0 000000018000532c f   WindowsNativeDispatcher.obj
 0001:00004358       Java_sun_nio_fs_WindowsNativeDispatcher_DeviceIoControlGetReparsePoint 0000000180005358 f   WindowsNativeDispatcher.obj
 0001:000043b0       Java_sun_nio_fs_WindowsNativeDispatcher_DeviceIoControlSetSparse 00000001800053b0 f   WindowsNativeDispatcher.obj
 0001:00004404       Java_sun_nio_fs_WindowsNativeDispatcher_DuplicateTokenEx 0000000180005404 f   WindowsNativeDispatcher.obj
 0001:00004454       Java_sun_nio_fs_WindowsNativeDispatcher_FindClose 0000000180005454 f   WindowsNativeDispatcher.obj
 0001:00004480       Java_sun_nio_fs_WindowsNativeDispatcher_FindFirstFile0 0000000180005480 f   WindowsNativeDispatcher.obj
 0001:0000456c       Java_sun_nio_fs_WindowsNativeDispatcher_FindFirstFile1 000000018000556c f   WindowsNativeDispatcher.obj
 0001:000045ac       Java_sun_nio_fs_WindowsNativeDispatcher_FindFirstStream0 00000001800055ac f   WindowsNativeDispatcher.obj
 0001:000046ac       Java_sun_nio_fs_WindowsNativeDispatcher_FindNextFile 00000001800056ac f   WindowsNativeDispatcher.obj
 0001:00004720       Java_sun_nio_fs_WindowsNativeDispatcher_FindNextStream 0000000180005720 f   WindowsNativeDispatcher.obj
 0001:000047b4       Java_sun_nio_fs_WindowsNativeDispatcher_GetAce 00000001800057b4 f   WindowsNativeDispatcher.obj
 0001:000047f4       Java_sun_nio_fs_WindowsNativeDispatcher_GetAclInformation0 00000001800057f4 f   WindowsNativeDispatcher.obj
 0001:00004878       Java_sun_nio_fs_WindowsNativeDispatcher_GetCurrentProcess 0000000180005878 f   WindowsNativeDispatcher.obj
 0001:00004880       Java_sun_nio_fs_WindowsNativeDispatcher_GetCurrentThread 0000000180005880 f   WindowsNativeDispatcher.obj
 0001:00004888       Java_sun_nio_fs_WindowsNativeDispatcher_GetDiskFreeSpace0 0000000180005888 f   WindowsNativeDispatcher.obj
 0001:000048f8       Java_sun_nio_fs_WindowsNativeDispatcher_GetDiskFreeSpaceEx0 00000001800058f8 f   WindowsNativeDispatcher.obj
 0001:00004994       Java_sun_nio_fs_WindowsNativeDispatcher_GetDriveType0 0000000180005994 f   WindowsNativeDispatcher.obj
 0001:000049a0       Java_sun_nio_fs_WindowsNativeDispatcher_GetFileAttributes0 00000001800059a0 f   WindowsNativeDispatcher.obj
 0001:000049dc       Java_sun_nio_fs_WindowsNativeDispatcher_GetFileAttributesEx0 00000001800059dc f   WindowsNativeDispatcher.obj
 0001:00004a10       Java_sun_nio_fs_WindowsNativeDispatcher_GetFileInformationByHandle 0000000180005a10 f   WindowsNativeDispatcher.obj
 0001:00004a40       Java_sun_nio_fs_WindowsNativeDispatcher_GetFileSecurity0 0000000180005a40 f   WindowsNativeDispatcher.obj
 0001:00004aa4       Java_sun_nio_fs_WindowsNativeDispatcher_GetFinalPathNameByHandle 0000000180005aa4 f   WindowsNativeDispatcher.obj
 0001:00004bbc       Java_sun_nio_fs_WindowsNativeDispatcher_GetFullPathName0 0000000180005bbc f   WindowsNativeDispatcher.obj
 0001:00004cd0       Java_sun_nio_fs_WindowsNativeDispatcher_GetLengthSid 0000000180005cd0 f   WindowsNativeDispatcher.obj
 0001:00004cdc       Java_sun_nio_fs_WindowsNativeDispatcher_GetLogicalDrives 0000000180005cdc f   WindowsNativeDispatcher.obj
 0001:00004d14       Java_sun_nio_fs_WindowsNativeDispatcher_GetOverlappedResult 0000000180005d14 f   WindowsNativeDispatcher.obj
 0001:00004d5c       Java_sun_nio_fs_WindowsNativeDispatcher_GetQueuedCompletionStatus0 0000000180005d5c f   WindowsNativeDispatcher.obj
 0001:00004e0c       Java_sun_nio_fs_WindowsNativeDispatcher_GetSecurityDescriptorDacl 0000000180005e0c f   WindowsNativeDispatcher.obj
 0001:00004e5c       Java_sun_nio_fs_WindowsNativeDispatcher_GetSecurityDescriptorOwner 0000000180005e5c f   WindowsNativeDispatcher.obj
 0001:00004e9c       Java_sun_nio_fs_WindowsNativeDispatcher_GetTokenInformation 0000000180005e9c f   WindowsNativeDispatcher.obj
 0001:00004efc       Java_sun_nio_fs_WindowsNativeDispatcher_GetVolumeInformation0 0000000180005efc f   WindowsNativeDispatcher.obj
 0001:00005054       Java_sun_nio_fs_WindowsNativeDispatcher_GetVolumePathName0 0000000180006054 f   WindowsNativeDispatcher.obj
 0001:000050e8       Java_sun_nio_fs_WindowsNativeDispatcher_InitializeAcl 00000001800060e8 f   WindowsNativeDispatcher.obj
 0001:00005120       Java_sun_nio_fs_WindowsNativeDispatcher_InitializeSecurityDescriptor 0000000180006120 f   WindowsNativeDispatcher.obj
 0001:00005154       Java_sun_nio_fs_WindowsNativeDispatcher_LocalFree 0000000180006154 f   WindowsNativeDispatcher.obj
 0001:00005160       Java_sun_nio_fs_WindowsNativeDispatcher_LookupAccountName0 0000000180006160 f   WindowsNativeDispatcher.obj
 0001:000051fc       Java_sun_nio_fs_WindowsNativeDispatcher_LookupAccountSid0 00000001800061fc f   WindowsNativeDispatcher.obj
 0001:00005344       Java_sun_nio_fs_WindowsNativeDispatcher_LookupPrivilegeValue0 0000000180006344 f   WindowsNativeDispatcher.obj
 0001:000053b4       Java_sun_nio_fs_WindowsNativeDispatcher_MoveFileEx0 00000001800063b4 f   WindowsNativeDispatcher.obj
 0001:000053ec       Java_sun_nio_fs_WindowsNativeDispatcher_OpenProcessToken 00000001800063ec f   WindowsNativeDispatcher.obj
 0001:00005428       Java_sun_nio_fs_WindowsNativeDispatcher_OpenThreadToken 0000000180006428 f   WindowsNativeDispatcher.obj
 0001:00005484       Java_sun_nio_fs_WindowsNativeDispatcher_PostQueuedCompletionStatus 0000000180006484 f   WindowsNativeDispatcher.obj
 0001:000054c0       Java_sun_nio_fs_WindowsNativeDispatcher_ReadDirectoryChangesW 00000001800064c0 f   WindowsNativeDispatcher.obj
 0001:00005530       Java_sun_nio_fs_WindowsNativeDispatcher_RemoveDirectory0 0000000180006530 f   WindowsNativeDispatcher.obj
 0001:0000555c       Java_sun_nio_fs_WindowsNativeDispatcher_SetEndOfFile 000000018000655c f   WindowsNativeDispatcher.obj
 0001:00005588       Java_sun_nio_fs_WindowsNativeDispatcher_SetFileAttributes0 0000000180006588 f   WindowsNativeDispatcher.obj
 0001:000055b8       Java_sun_nio_fs_WindowsNativeDispatcher_SetFileSecurity0 00000001800065b8 f   WindowsNativeDispatcher.obj
 0001:000055f0       Java_sun_nio_fs_WindowsNativeDispatcher_SetFileTime 00000001800065f0 f   WindowsNativeDispatcher.obj
 0001:0000565c       Java_sun_nio_fs_WindowsNativeDispatcher_SetSecurityDescriptorDacl 000000018000665c f   WindowsNativeDispatcher.obj
 0001:00005698       Java_sun_nio_fs_WindowsNativeDispatcher_SetSecurityDescriptorOwner 0000000180006698 f   WindowsNativeDispatcher.obj
 0001:000056d0       Java_sun_nio_fs_WindowsNativeDispatcher_SetThreadToken 00000001800066d0 f   WindowsNativeDispatcher.obj
 0001:00005700       Java_sun_nio_fs_WindowsNativeDispatcher_initIDs 0000000180006700 f   WindowsNativeDispatcher.obj
 0001:00005b68       Java_sun_nio_ch_WindowsSelectorImpl_00024SubSelector_poll0 0000000180006b68 f   WindowsSelectorImpl.obj
 0001:00005f40       Java_sun_nio_ch_WindowsSelectorImpl_discardUrgentData 0000000180006f40 f   WindowsSelectorImpl.obj
 0001:00005f98       Java_sun_nio_ch_WindowsSelectorImpl_resetWakeupSocket0 0000000180006f98 f   WindowsSelectorImpl.obj
 0001:00006050       Java_sun_nio_ch_WindowsSelectorImpl_setWakeupSocket0 0000000180007050 f   WindowsSelectorImpl.obj
 0001:00006074       JNI_OnLoad                 0000000180007074 f   nio_util.obj
 0001:0000609c       __WSAFDIsSet               000000018000709c f   ws2_32:WS2_32.dll
 0001:000060a2       JNU_ThrowByName            00000001800070a2 f   java:java.dll
 0001:000060a8       JNU_ThrowOutOfMemoryError  00000001800070a8 f   java:java.dll
 0001:000060ae       JNU_ThrowIOExceptionWithLastError 00000001800070ae f   java:java.dll
 0001:000060b4       Java_sun_security_provider_NativeSeedGenerator_nativeGenerateSeed 00000001800070b4 f   java:java.dll
 0001:000060ba       JNU_ThrowInternalError     00000001800070ba f   java:java.dll
 0001:000060c0       JNU_NewObjectByName        00000001800070c0 f   java:java.dll
 0001:000060c6       NET_InetAddressToSockaddr  00000001800070c6 f   net:net.dll
 0001:000060cc       NET_SockaddrToInetAddress  00000001800070cc f   net:net.dll
 0001:000060d2       NET_GetPortFromSockaddr    00000001800070d2 f   net:net.dll
 0001:000060d8       NET_SockaddrEqualsInetAddress 00000001800070d8 f   net:net.dll
 0001:000060de       NET_WinBind                00000001800070de f   net:net.dll
 0001:000060e4       NET_EnableFastTcpLoopbackConnect 00000001800070e4 f   net:net.dll
 0001:000060ea       initInetAddressIDs         00000001800070ea f   net:net.dll
 0001:000060f0       NET_ThrowNew               00000001800070f0 f   net:net.dll
 0001:000060f6       ipv6_available             00000001800070f6 f   net:net.dll
 0001:000060fc       NET_GetSockOpt             00000001800070fc f   net:net.dll
 0001:00006102       NET_SetSockOpt             0000000180007102 f   net:net.dll
 0001:00006108       NET_EnableFastTcpLoopback  0000000180007108 f   net:net.dll
 0001:0000610e       ConvertSidToStringSidW     000000018000710e f   advapi32:ADVAPI32.dll
 0001:00006114       ConvertStringSidToSidW     0000000180007114 f   advapi32:ADVAPI32.dll
 0001:0000611c       __GSHandlerCheck           000000018000711c f   MSVCRT:gshandler.obj
 0001:0000613c       __GSHandlerCheckCommon     000000018000713c f   MSVCRT:gshandler.obj
 0001:000061b0       __security_check_cookie    00000001800071b0 f   MSVCRT:amdsecgs.obj
 0001:000061e0       __chkstk                   00000001800071e0 f   MSVCRT:chkstk.obj
 0001:000061e0       _alloca_probe              00000001800071e0 f   MSVCRT:chkstk.obj
 0001:00006550       _DllMainCRTStartup         0000000180007550 f   MSVCRT:dll_dllmain.obj
 0001:00006590       __raise_securityfailure    0000000180007590 f   MSVCRT:gs_report.obj
 0001:000065c4       __report_gsfailure         00000001800075c4 f   MSVCRT:gs_report.obj
 0001:0000670c       __security_init_cookie     000000018000770c f   MSVCRT:gs_support.obj
 0001:000067b8       DllMain                    00000001800077b8 f   MSVCRT:dll_dllmain_stub.obj
 0001:000067dc       ?__scrt_initialize_type_info@@YAXXZ 00000001800077dc f   MSVCRT:tncleanup.obj
 0001:000067ec       ?__scrt_uninitialize_type_info@@YAXXZ 00000001800077ec f   MSVCRT:tncleanup.obj
 0001:000067f8       __local_stdio_printf_options 00000001800077f8 f i MSVCRT:default_local_stdio_options.obj
 0001:00006800       __local_stdio_scanf_options 0000000180007800 f i MSVCRT:default_local_stdio_options.obj
 0001:00006808       __scrt_initialize_default_local_stdio_options 0000000180007808 f   MSVCRT:default_local_stdio_options.obj
 0001:00006824       __scrt_acquire_startup_lock 0000000180007824 f   MSVCRT:utility.obj
 0001:00006860       __scrt_dllmain_after_initialize_c 0000000180007860 f   MSVCRT:utility.obj
 0001:00006894       __scrt_dllmain_before_initialize_c 0000000180007894 f   MSVCRT:utility.obj
 0001:000068ac       __scrt_dllmain_crt_thread_attach 00000001800078ac f   MSVCRT:utility.obj
 0001:000068d4       __scrt_dllmain_crt_thread_detach 00000001800078d4 f   MSVCRT:utility.obj
 0001:000068ec       __scrt_dllmain_exception_filter 00000001800078ec f   MSVCRT:utility.obj
 0001:0000694c       __scrt_dllmain_uninitialize_c 000000018000794c f   MSVCRT:utility.obj
 0001:0000697c       __scrt_dllmain_uninitialize_critical 000000018000797c f   MSVCRT:utility.obj
 0001:00006990       __scrt_initialize_crt      0000000180007990 f   MSVCRT:utility.obj
 0001:000069dc       __scrt_initialize_onexit_tables 00000001800079dc f   MSVCRT:utility.obj
 0001:00006a68       __scrt_is_nonwritable_in_current_image 0000000180007a68 f   MSVCRT:utility.obj
 0001:00006b00       __scrt_release_startup_lock 0000000180007b00 f   MSVCRT:utility.obj
 0001:00006b24       __scrt_uninitialize_crt    0000000180007b24 f   MSVCRT:utility.obj
 0001:00006b50       __scrt_get_dyn_tls_init_callback 0000000180007b50 f   MSVCRT:dyn_tls_init.obj
 0001:00006b58       __crt_debugger_hook        0000000180007b58 f   MSVCRT:utility_desktop.obj
 0001:00006b60       __scrt_fastfail            0000000180007b60 f   MSVCRT:utility_desktop.obj
 0001:00006cac       _RTC_Initialize            0000000180007cac f   MSVCRT:initsect.obj
 0001:00006ce8       _RTC_Terminate             0000000180007ce8 f   MSVCRT:initsect.obj
 0001:00006d24       __isa_available_init       0000000180007d24 f   MSVCRT:cpu_disp.obj
 0001:00006ed0       __scrt_is_ucrt_dll_in_use  0000000180007ed0 f   MSVCRT:ucrt_detection.obj
 0001:00006ee0       TransmitFile               0000000180007ee0 f   Mswsock:MSWSOCK.dll
 0001:00006ee6       memset                     0000000180007ee6 f   vcruntime:VCRUNTIME140.dll
 0001:00006eec       __C_specific_handler       0000000180007eec f   vcruntime:VCRUNTIME140.dll
 0001:00006ef2       __std_type_info_destroy_list 0000000180007ef2 f   vcruntime:VCRUNTIME140.dll
 0001:00006ef8       _initterm                  0000000180007ef8 f   ucrt:api-ms-win-crt-runtime-l1-1-0.dll
 0001:00006efe       _initterm_e                0000000180007efe f   ucrt:api-ms-win-crt-runtime-l1-1-0.dll
 0001:00006f04       _seh_filter_dll            0000000180007f04 f   ucrt:api-ms-win-crt-runtime-l1-1-0.dll
 0001:00006f0a       _configure_narrow_argv     0000000180007f0a f   ucrt:api-ms-win-crt-runtime-l1-1-0.dll
 0001:00006f10       _initialize_narrow_environment 0000000180007f10 f   ucrt:api-ms-win-crt-runtime-l1-1-0.dll
 0001:00006f16       _initialize_onexit_table   0000000180007f16 f   ucrt:api-ms-win-crt-runtime-l1-1-0.dll
 0001:00006f1c       _execute_onexit_table      0000000180007f1c f   ucrt:api-ms-win-crt-runtime-l1-1-0.dll
 0001:00006f22       _cexit                     0000000180007f22 f   ucrt:api-ms-win-crt-runtime-l1-1-0.dll
 0001:00006f28       __acrt_initialize          0000000180007f28 f   MSVCRT:ucrt_stubs.obj
 0001:00006f28       __acrt_thread_attach       0000000180007f28 f   MSVCRT:ucrt_stubs.obj
 0001:00006f28       __acrt_thread_detach       0000000180007f28 f   MSVCRT:ucrt_stubs.obj
 0001:00006f28       __acrt_uninitialize        0000000180007f28 f   MSVCRT:ucrt_stubs.obj
 0001:00006f28       __acrt_uninitialize_critical 0000000180007f28 f   MSVCRT:ucrt_stubs.obj
 0001:00006f28       __scrt_stub_for_acrt_initialize 0000000180007f28 f   MSVCRT:ucrt_stubs.obj
 0001:00006f28       __scrt_stub_for_acrt_thread_attach 0000000180007f28 f   MSVCRT:ucrt_stubs.obj
 0001:00006f28       __scrt_stub_for_acrt_thread_detach 0000000180007f28 f   MSVCRT:ucrt_stubs.obj
 0001:00006f28       __scrt_stub_for_acrt_uninitialize 0000000180007f28 f   MSVCRT:ucrt_stubs.obj
 0001:00006f28       __scrt_stub_for_acrt_uninitialize_critical 0000000180007f28 f   MSVCRT:ucrt_stubs.obj
 0001:00006f28       __vcrt_initialize          0000000180007f28 f   MSVCRT:ucrt_stubs.obj
 0001:00006f28       __vcrt_thread_attach       0000000180007f28 f   MSVCRT:ucrt_stubs.obj
 0001:00006f28       __vcrt_thread_detach       0000000180007f28 f   MSVCRT:ucrt_stubs.obj
 0001:00006f28       __vcrt_uninitialize        0000000180007f28 f   MSVCRT:ucrt_stubs.obj
 0001:00006f28       __vcrt_uninitialize_critical 0000000180007f28 f   MSVCRT:ucrt_stubs.obj
 0001:00006f2c       __scrt_stub_for_is_c_termination_complete 0000000180007f2c f   MSVCRT:ucrt_stubs.obj
 0001:00006f2c       _is_c_termination_complete 0000000180007f2c f   MSVCRT:ucrt_stubs.obj
 0001:00006f2f       memcpy                     0000000180007f2f f   vcruntime:VCRUNTIME140.dll
 0001:00006f50       _guard_dispatch_icall_nop  0000000180007f50 f   MSVCRT:guard_dispatch.obj
 0001:00006f70       _guard_xfg_dispatch_icall_nop 0000000180007f70 f   MSVCRT:guard_xfg_dispatch.obj
 0002:00000000       __imp_GetAce               0000000180009000     advapi32:ADVAPI32.dll
 0002:00000008       __imp_ConvertStringSidToSidW 0000000180009008     advapi32:ADVAPI32.dll
 0002:00000010       __imp_ConvertSidToStringSidW 0000000180009010     advapi32:ADVAPI32.dll
 0002:00000018       __imp_LookupPrivilegeValueW 0000000180009018     advapi32:ADVAPI32.dll
 0002:00000020       __imp_LookupAccountNameW   0000000180009020     advapi32:ADVAPI32.dll
 0002:00000028       __imp_LookupAccountSidW    0000000180009028     advapi32:ADVAPI32.dll
 0002:00000030       __imp_SetSecurityDescriptorOwner 0000000180009030     advapi32:ADVAPI32.dll
 0002:00000038       __imp_SetSecurityDescriptorDacl 0000000180009038     advapi32:ADVAPI32.dll
 0002:00000040       __imp_SetFileSecurityW     0000000180009040     advapi32:ADVAPI32.dll
 0002:00000048       __imp_MapGenericMask       0000000180009048     advapi32:ADVAPI32.dll
 0002:00000050       __imp_InitializeSecurityDescriptor 0000000180009050     advapi32:ADVAPI32.dll
 0002:00000058       __imp_InitializeAcl        0000000180009058     advapi32:ADVAPI32.dll
 0002:00000060       __imp_GetTokenInformation  0000000180009060     advapi32:ADVAPI32.dll
 0002:00000068       __imp_GetSecurityDescriptorOwner 0000000180009068     advapi32:ADVAPI32.dll
 0002:00000070       __imp_GetSecurityDescriptorDacl 0000000180009070     advapi32:ADVAPI32.dll
 0002:00000078       __imp_GetLengthSid         0000000180009078     advapi32:ADVAPI32.dll
 0002:00000080       __imp_GetFileSecurityW     0000000180009080     advapi32:ADVAPI32.dll
 0002:00000088       __imp_GetAclInformation    0000000180009088     advapi32:ADVAPI32.dll
 0002:00000090       __imp_DuplicateTokenEx     0000000180009090     advapi32:ADVAPI32.dll
 0002:00000098       __imp_AdjustTokenPrivileges 0000000180009098     advapi32:ADVAPI32.dll
 0002:000000a0       __imp_AddAccessDeniedAceEx 00000001800090a0     advapi32:ADVAPI32.dll
 0002:000000a8       __imp_AddAccessAllowedAceEx 00000001800090a8     advapi32:ADVAPI32.dll
 0002:000000b0       __imp_AccessCheck          00000001800090b0     advapi32:ADVAPI32.dll
 0002:000000b8       __imp_OpenThreadToken      00000001800090b8     advapi32:ADVAPI32.dll
 0002:000000c0       __imp_OpenProcessToken     00000001800090c0     advapi32:ADVAPI32.dll
 0002:000000c8       __imp_SetThreadToken       00000001800090c8     advapi32:ADVAPI32.dll
 0002:000000d0       __imp_RegQueryValueExW     00000001800090d0     advapi32:ADVAPI32.dll
 0002:000000d8       __imp_RegOpenKeyExW        00000001800090d8     advapi32:ADVAPI32.dll
 0002:000000e0       __imp_RegCloseKey          00000001800090e0     advapi32:ADVAPI32.dll
 0002:000000e8       \177ADVAPI32_NULL_THUNK_DATA 00000001800090e8     advapi32:ADVAPI32.dll
 0002:000000f0       __imp_GetCurrentThread     00000001800090f0     kernel32:KERNEL32.dll
 0002:000000f8       __imp_CreateEventW         00000001800090f8     kernel32:KERNEL32.dll
 0002:00000100       __imp_CancelIo             0000000180009100     kernel32:KERNEL32.dll
 0002:00000108       __imp_DeviceIoControl      0000000180009108     kernel32:KERNEL32.dll
 0002:00000110       __imp_FindNextStreamW      0000000180009110     kernel32:KERNEL32.dll
 0002:00000118       __imp_FindFirstStreamW     0000000180009118     kernel32:KERNEL32.dll
 0002:00000120       __imp_SetFileTime          0000000180009120     kernel32:KERNEL32.dll
 0002:00000128       __imp_LocalAlloc           0000000180009128     kernel32:KERNEL32.dll
 0002:00000130       __imp_SetEndOfFile         0000000180009130     kernel32:KERNEL32.dll
 0002:00000138       __imp_RemoveDirectoryW     0000000180009138     kernel32:KERNEL32.dll
 0002:00000140       __imp_GetVolumePathNameW   0000000180009140     kernel32:KERNEL32.dll
 0002:00000148       __imp_GetVolumeInformationW 0000000180009148     kernel32:KERNEL32.dll
 0002:00000150       __imp_GetLogicalDrives     0000000180009150     kernel32:KERNEL32.dll
 0002:00000158       __imp_GetFullPathNameW     0000000180009158     kernel32:KERNEL32.dll
 0002:00000160       __imp_GetFinalPathNameByHandleW 0000000180009160     kernel32:KERNEL32.dll
 0002:00000168       __imp_LocalFree            0000000180009168     kernel32:KERNEL32.dll
 0002:00000170       __imp_CopyFileExW          0000000180009170     kernel32:KERNEL32.dll
 0002:00000178       __imp_MoveFileExW          0000000180009178     kernel32:KERNEL32.dll
 0002:00000180       __imp_CreateHardLinkW      0000000180009180     kernel32:KERNEL32.dll
 0002:00000188       __imp_ReadDirectoryChangesW 0000000180009188     kernel32:KERNEL32.dll
 0002:00000190       __imp_CreateSymbolicLinkW  0000000180009190     kernel32:KERNEL32.dll
 0002:00000198       __imp_RtlCaptureContext    0000000180009198     kernel32:KERNEL32.dll
 0002:000001a0       __imp_RtlLookupFunctionEntry 00000001800091a0     kernel32:KERNEL32.dll
 0002:000001a8       __imp_RtlVirtualUnwind     00000001800091a8     kernel32:KERNEL32.dll
 0002:000001b0       __imp_UnhandledExceptionFilter 00000001800091b0     kernel32:KERNEL32.dll
 0002:000001b8       __imp_SetUnhandledExceptionFilter 00000001800091b8     kernel32:KERNEL32.dll
 0002:000001c0       __imp_UnlockFileEx         00000001800091c0     kernel32:KERNEL32.dll
 0002:000001c8       __imp_TerminateProcess     00000001800091c8     kernel32:KERNEL32.dll
 0002:000001d0       __imp_IsProcessorFeaturePresent 00000001800091d0     kernel32:KERNEL32.dll
 0002:000001d8       __imp_QueryPerformanceCounter 00000001800091d8     kernel32:KERNEL32.dll
 0002:000001e0       __imp_GetCurrentProcessId  00000001800091e0     kernel32:KERNEL32.dll
 0002:000001e8       __imp_GetCurrentThreadId   00000001800091e8     kernel32:KERNEL32.dll
 0002:000001f0       __imp_GetSystemTimeAsFileTime 00000001800091f0     kernel32:KERNEL32.dll
 0002:000001f8       __imp_DisableThreadLibraryCalls 00000001800091f8     kernel32:KERNEL32.dll
 0002:00000200       __imp_InitializeSListHead  0000000180009200     kernel32:KERNEL32.dll
 0002:00000208       __imp_IsDebuggerPresent    0000000180009208     kernel32:KERNEL32.dll
 0002:00000210       __imp_FindClose            0000000180009210     kernel32:KERNEL32.dll
 0002:00000218       __imp_FindFirstFileW       0000000180009218     kernel32:KERNEL32.dll
 0002:00000220       __imp_FindNextFileW        0000000180009220     kernel32:KERNEL32.dll
 0002:00000228       __imp_GetDiskFreeSpaceExW  0000000180009228     kernel32:KERNEL32.dll
 0002:00000230       __imp_GetDriveTypeW        0000000180009230     kernel32:KERNEL32.dll
 0002:00000238       __imp_GetFileAttributesW   0000000180009238     kernel32:KERNEL32.dll
 0002:00000240       __imp_SetFileAttributesW   0000000180009240     kernel32:KERNEL32.dll
 0002:00000248       __imp_DeleteFileW          0000000180009248     kernel32:KERNEL32.dll
 0002:00000250       __imp_CreateFileW          0000000180009250     kernel32:KERNEL32.dll
 0002:00000258       __imp_SetFilePointerEx     0000000180009258     kernel32:KERNEL32.dll
 0002:00000260       __imp_CloseHandle          0000000180009260     kernel32:KERNEL32.dll
 0002:00000268       __imp_GetLastError         0000000180009268     kernel32:KERNEL32.dll
 0002:00000270       __imp_GetSystemInfo        0000000180009270     kernel32:KERNEL32.dll
 0002:00000278       __imp_MapViewOfFile        0000000180009278     kernel32:KERNEL32.dll
 0002:00000280       __imp_UnmapViewOfFile      0000000180009280     kernel32:KERNEL32.dll
 0002:00000288       __imp_CreateFileMappingA   0000000180009288     kernel32:KERNEL32.dll
 0002:00000290       __imp_FlushFileBuffers     0000000180009290     kernel32:KERNEL32.dll
 0002:00000298       __imp_GetDiskFreeSpaceW    0000000180009298     kernel32:KERNEL32.dll
 0002:000002a0       __imp_GetFileSizeEx        00000001800092a0     kernel32:KERNEL32.dll
 0002:000002a8       __imp_LockFileEx           00000001800092a8     kernel32:KERNEL32.dll
 0002:000002b0       __imp_ReadFile             00000001800092b0     kernel32:KERNEL32.dll
 0002:000002b8       __imp_SetFileInformationByHandle 00000001800092b8     kernel32:KERNEL32.dll
 0002:000002c0       __imp_CreateDirectoryW     00000001800092c0     kernel32:KERNEL32.dll
 0002:000002c8       __imp_WriteFile            00000001800092c8     kernel32:KERNEL32.dll
 0002:000002d0       __imp_DuplicateHandle      00000001800092d0     kernel32:KERNEL32.dll
 0002:000002d8       __imp_GetOverlappedResult  00000001800092d8     kernel32:KERNEL32.dll
 0002:000002e0       __imp_GetCurrentProcess    00000001800092e0     kernel32:KERNEL32.dll
 0002:000002e8       __imp_ReOpenFile           00000001800092e8     kernel32:KERNEL32.dll
 0002:000002f0       __imp_GetFileInformationByHandle 00000001800092f0     kernel32:KERNEL32.dll
 0002:000002f8       __imp_CreateIoCompletionPort 00000001800092f8     kernel32:KERNEL32.dll
 0002:00000300       __imp_GetQueuedCompletionStatus 0000000180009300     kernel32:KERNEL32.dll
 0002:00000308       __imp_PostQueuedCompletionStatus 0000000180009308     kernel32:KERNEL32.dll
 0002:00000310       __imp_FormatMessageW       0000000180009310     kernel32:KERNEL32.dll
 0002:00000318       __imp_FlushViewOfFile      0000000180009318     kernel32:KERNEL32.dll
 0002:00000320       __imp_SetHandleInformation 0000000180009320     kernel32:KERNEL32.dll
 0002:00000328       __imp_GetFileAttributesExW 0000000180009328     kernel32:KERNEL32.dll
 0002:00000330       \177KERNEL32_NULL_THUNK_DATA 0000000180009330     kernel32:KERNEL32.dll
 0002:00000338       __imp_TransmitFile         0000000180009338     Mswsock:MSWSOCK.dll
 0002:00000340       \177MSWSOCK_NULL_THUNK_DATA 0000000180009340     Mswsock:MSWSOCK.dll
 0002:00000348       __imp_memset               0000000180009348     vcruntime:VCRUNTIME140.dll
 0002:00000350       __imp___C_specific_handler 0000000180009350     vcruntime:VCRUNTIME140.dll
 0002:00000358       __imp___std_type_info_destroy_list 0000000180009358     vcruntime:VCRUNTIME140.dll
 0002:00000360       __imp_memcpy               0000000180009360     vcruntime:VCRUNTIME140.dll
 0002:00000368       \177VCRUNTIME140_NULL_THUNK_DATA 0000000180009368     vcruntime:VCRUNTIME140.dll
 0002:00000370       __imp_getpeername          0000000180009370     ws2_32:WS2_32.dll
 0002:00000378       __imp_recvfrom             0000000180009378     ws2_32:WS2_32.dll
 0002:00000380       __imp_select               0000000180009380     ws2_32:WS2_32.dll
 0002:00000388       __imp_sendto               0000000180009388     ws2_32:WS2_32.dll
 0002:00000390       __imp_WSAGetLastError      0000000180009390     ws2_32:WS2_32.dll
 0002:00000398       __imp_WSAIoctl             0000000180009398     ws2_32:WS2_32.dll
 0002:000003a0       __imp_WSARecv              00000001800093a0     ws2_32:WS2_32.dll
 0002:000003a8       __imp_WSASend              00000001800093a8     ws2_32:WS2_32.dll
 0002:000003b0       __imp_ioctlsocket          00000001800093b0     ws2_32:WS2_32.dll
 0002:000003b8       __imp_WSAEventSelect       00000001800093b8     ws2_32:WS2_32.dll
 0002:000003c0       __imp___WSAFDIsSet         00000001800093c0     ws2_32:WS2_32.dll
 0002:000003c8       __imp_connect              00000001800093c8     ws2_32:WS2_32.dll
 0002:000003d0       __imp_getsockname          00000001800093d0     ws2_32:WS2_32.dll
 0002:000003d8       __imp_getsockopt           00000001800093d8     ws2_32:WS2_32.dll
 0002:000003e0       __imp_htonl                00000001800093e0     ws2_32:WS2_32.dll
 0002:000003e8       __imp_listen               00000001800093e8     ws2_32:WS2_32.dll
 0002:000003f0       __imp_ntohl                00000001800093f0     ws2_32:WS2_32.dll
 0002:000003f8       __imp_setsockopt           00000001800093f8     ws2_32:WS2_32.dll
 0002:00000400       __imp_shutdown             0000000180009400     ws2_32:WS2_32.dll
 0002:00000408       __imp_socket               0000000180009408     ws2_32:WS2_32.dll
 0002:00000410       __imp_recv                 0000000180009410     ws2_32:WS2_32.dll
 0002:00000418       __imp_closesocket          0000000180009418     ws2_32:WS2_32.dll
 0002:00000420       __imp_send                 0000000180009420     ws2_32:WS2_32.dll
 0002:00000428       __imp_accept               0000000180009428     ws2_32:WS2_32.dll
 0002:00000430       \177WS2_32_NULL_THUNK_DATA 0000000180009430     ws2_32:WS2_32.dll
 0002:00000438       __imp_malloc               0000000180009438     ucrt:api-ms-win-crt-heap-l1-1-0.dll
 0002:00000440       __imp_free                 0000000180009440     ucrt:api-ms-win-crt-heap-l1-1-0.dll
 0002:00000448       \177api-ms-win-crt-heap-l1-1-0_NULL_THUNK_DATA 0000000180009448     ucrt:api-ms-win-crt-heap-l1-1-0.dll
 0002:00000450       __imp__initterm            0000000180009450     ucrt:api-ms-win-crt-runtime-l1-1-0.dll
 0002:00000458       __imp__errno               0000000180009458     ucrt:api-ms-win-crt-runtime-l1-1-0.dll
 0002:00000460       __imp__configure_narrow_argv 0000000180009460     ucrt:api-ms-win-crt-runtime-l1-1-0.dll
 0002:00000468       __imp__initialize_narrow_environment 0000000180009468     ucrt:api-ms-win-crt-runtime-l1-1-0.dll
 0002:00000470       __imp__initialize_onexit_table 0000000180009470     ucrt:api-ms-win-crt-runtime-l1-1-0.dll
 0002:00000478       __imp__initterm_e          0000000180009478     ucrt:api-ms-win-crt-runtime-l1-1-0.dll
 0002:00000480       __imp__execute_onexit_table 0000000180009480     ucrt:api-ms-win-crt-runtime-l1-1-0.dll
 0002:00000488       __imp__cexit               0000000180009488     ucrt:api-ms-win-crt-runtime-l1-1-0.dll
 0002:00000490       __imp__seh_filter_dll      0000000180009490     ucrt:api-ms-win-crt-runtime-l1-1-0.dll
 0002:00000498       \177api-ms-win-crt-runtime-l1-1-0_NULL_THUNK_DATA 0000000180009498     ucrt:api-ms-win-crt-runtime-l1-1-0.dll
 0002:000004a0       __imp__get_osfhandle       00000001800094a0     ucrt:api-ms-win-crt-stdio-l1-1-0.dll
 0002:000004a8       \177api-ms-win-crt-stdio-l1-1-0_NULL_THUNK_DATA 00000001800094a8     ucrt:api-ms-win-crt-stdio-l1-1-0.dll
 0002:000004b0       __imp_wcslen               00000001800094b0     ucrt:api-ms-win-crt-string-l1-1-0.dll
 0002:000004b8       \177api-ms-win-crt-string-l1-1-0_NULL_THUNK_DATA 00000001800094b8     ucrt:api-ms-win-crt-string-l1-1-0.dll
 0002:000004c0       __imp_JNU_ThrowByName      00000001800094c0     java:java.dll
 0002:000004c8       __imp_JNU_NewObjectByName  00000001800094c8     java:java.dll
 0002:000004d0       __imp_JNU_ThrowInternalError 00000001800094d0     java:java.dll
 0002:000004d8       __imp_Java_sun_security_provider_NativeSeedGenerator_nativeGenerateSeed 00000001800094d8     java:java.dll
 0002:000004e0       __imp_JNU_ThrowIOExceptionWithLastError 00000001800094e0     java:java.dll
 0002:000004e8       __imp_JNU_ThrowOutOfMemoryError 00000001800094e8     java:java.dll
 0002:000004f0       \177java_NULL_THUNK_DATA   00000001800094f0     java:java.dll
 0002:000004f8       __imp_NET_SetSockOpt       00000001800094f8     net:net.dll
 0002:00000500       __imp_NET_GetSockOpt       0000000180009500     net:net.dll
 0002:00000508       __imp_ipv6_available       0000000180009508     net:net.dll
 0002:00000510       __imp_NET_ThrowNew         0000000180009510     net:net.dll
 0002:00000518       __imp_initInetAddressIDs   0000000180009518     net:net.dll
 0002:00000520       __imp_NET_EnableFastTcpLoopbackConnect 0000000180009520     net:net.dll
 0002:00000528       __imp_NET_WinBind          0000000180009528     net:net.dll
 0002:00000530       __imp_NET_SockaddrEqualsInetAddress 0000000180009530     net:net.dll
 0002:00000538       __imp_NET_GetPortFromSockaddr 0000000180009538     net:net.dll
 0002:00000540       __imp_NET_SockaddrToInetAddress 0000000180009540     net:net.dll
 0002:00000548       __imp_NET_InetAddressToSockaddr 0000000180009548     net:net.dll
 0002:00000550       __imp_NET_EnableFastTcpLoopback 0000000180009550     net:net.dll
 0002:00000558       \177net_NULL_THUNK_DATA    0000000180009558     net:net.dll
 0002:00000560       __guard_check_icall_fptr   0000000180009560     MSVCRT:guard_support.obj
 0002:00000568       __guard_xfg_check_icall_fptr 0000000180009568     MSVCRT:guard_support.obj
 0002:00000570       __guard_dispatch_icall_fptr 0000000180009570     MSVCRT:guard_support.obj
 0002:00000578       __guard_xfg_dispatch_icall_fptr 0000000180009578     MSVCRT:guard_support.obj
 0002:00000580       __guard_xfg_table_dispatch_icall_fptr 0000000180009580     MSVCRT:guard_support.obj
 0002:00000588       __castguard_check_failure_os_handled_fptr 0000000180009588     MSVCRT:guard_support.obj
 0002:00000590       __guard_memcpy_fptr        0000000180009590     vcruntime:softmemtag.obj
 0002:00000598       __xc_a                     0000000180009598     MSVCRT:initializers.obj
 0002:000005a0       __xc_z                     00000001800095a0     MSVCRT:initializers.obj
 0002:000005a8       __xi_a                     00000001800095a8     MSVCRT:initializers.obj
 0002:000005b0       __xi_z                     00000001800095b0     MSVCRT:initializers.obj
 0002:000005b8       __xp_a                     00000001800095b8     MSVCRT:initializers.obj
 0002:000005c0       __xp_z                     00000001800095c0     MSVCRT:initializers.obj
 0002:000005c8       __xt_a                     00000001800095c8     MSVCRT:initializers.obj
 0002:000005d0       __xt_z                     00000001800095d0     MSVCRT:initializers.obj
 0002:000005e0       ??_C@_0BL@HBNNAPLM@java?1net?1InetSocketAddress@ 00000001800095e0     DatagramChannelImpl.obj
 0002:00000600       ??_C@_0BL@KCCEIBDI@?$CILjava?1net?1InetAddress?$DLI?$CJV@ 0000000180009600     DatagramChannelImpl.obj
 0002:0000061c       ??_C@_06FALKBLGB@?$DMinit?$DO@ 000000018000961c     DatagramChannelImpl.obj
 0002:00000628       ??_C@_0BP@BNFFMBJL@sun?1nio?1ch?1DatagramChannelImpl@ 0000000180009628     DatagramChannelImpl.obj
 0002:00000648       ??_C@_0BJ@NDFGGFKE@Ljava?1net?1SocketAddress?$DL@ 0000000180009648     DatagramChannelImpl.obj
 0002:00000664       ??_C@_06CGHJMPBJ@sender@   0000000180009664     DatagramChannelImpl.obj
 0002:00000670       ??_C@_0BH@FIKCFBLO@Ljava?1net?1InetAddress?$DL@ 0000000180009670     DatagramChannelImpl.obj
 0002:00000688       ??_C@_0BI@OANHFGOF@cachedSenderInetAddress@ 0000000180009688     DatagramChannelImpl.obj
 0002:000006a0       ??_C@_01JPJNBJEM@I@        00000001800096a0     DatagramChannelImpl.obj
 0002:000006a8       ??_C@_0BB@JLIPPJNN@cachedSenderPort@ 00000001800096a8     DatagramChannelImpl.obj
 0002:000006c0       ??_C@_0CC@BDDMPFBF@java?1net?1PortUnreachableExcepti@ 00000001800096c0     DatagramChannelImpl.obj
 0002:000006e8       ??_C@_0P@DGIIHHAE@WSARecv?5failed@ 00000001800096e8     DatagramDispatcher.obj
 0002:000006f8       ??_C@_0P@NKOFNKCM@WSASend?5failed@ 00000001800096f8     DatagramDispatcher.obj
 0002:00000708       ??_C@_0BJ@BDFOFHPL@Ljava?1io?1FileDescriptor?$DL@ 0000000180009708     FileChannelImpl.obj
 0002:00000724       ??_C@_02ENHFDPNM@fd@       0000000180009724     FileChannelImpl.obj
 0002:00000728       ??_C@_0L@DPMFILPJ@Map?5failed@ 0000000180009728     FileChannelImpl.obj
 0002:00000738       ??_C@_0N@IGMMIDE@Unmap?5failed@ 0000000180009738     FileChannelImpl.obj
 0002:00000748       ??_C@_0BI@ICELLBHO@SetFilePointerEx?5failed@ 0000000180009748     FileChannelImpl.obj
 0002:00000760       ??_C@_0BA@CJMHIODJ@transfer?5failed@ 0000000180009760     FileChannelImpl.obj
 0002:00000770       ??_C@_0P@EFDAIKIF@Invalid?5handle@ 0000000180009770     FileDispatcherImpl.obj
 0002:00000780       ??_C@_0M@DCKEEFAG@Read?5failed@ 0000000180009780     FileDispatcherImpl.obj
 0002:00000790       ??_C@_0M@HPFDGGMC@Seek?5failed@ 0000000180009790     FileDispatcherImpl.obj
 0002:000007a0       ??_C@_0N@PGCLODBC@Write?5failed@ 00000001800097a0     FileDispatcherImpl.obj
 0002:000007b0       ??_C@_0N@EFKIKJEB@Force?5failed@ 00000001800097b0     FileDispatcherImpl.obj
 0002:000007c0       ??_C@_0BC@FODOCFKM@Truncation?5failed@ 00000001800097c0     FileDispatcherImpl.obj
 0002:000007d8       ??_C@_0M@GLCOPFPC@Size?5failed@ 00000001800097d8     FileDispatcherImpl.obj
 0002:000007e8       ??_C@_0M@OOGODMIM@Lock?5failed@ 00000001800097e8     FileDispatcherImpl.obj
 0002:000007f8       ??_C@_0P@MAMCLOFD@Release?5failed@ 00000001800097f8     FileDispatcherImpl.obj
 0002:00000808       ??_C@_0N@GNNFMAIG@Close?5failed@ 0000000180009808     FileDispatcherImpl.obj
 0002:00000818       ??_C@_0BH@OPJFPPPK@DuplicateHandle?5failed@ 0000000180009818     FileDispatcherImpl.obj
 0002:00000830       ??_C@_0BG@JDMBHIAK@DirectIO?5setup?5failed@ 0000000180009830     FileDispatcherImpl.obj
 0002:00000848       ??_C@_01LELAEKIP@J@        0000000180009848     FileKey.obj
 0002:00000850       ??_C@_0BF@GJBBDEBO@dwVolumeSerialNumber@ 0000000180009850     FileKey.obj
 0002:00000868       ??_C@_0P@OJOGHFHE@nFileIndexHigh@ 0000000180009868     FileKey.obj
 0002:00000878       ??_C@_0O@HJEFBNI@nFileIndexLow@ 0000000180009878     FileKey.obj
 0002:00000888       ??_C@_0CC@EJDNCKME@GetFileInformationByHandle?5fail@ 0000000180009888     FileKey.obj
 0002:000008b0       ??_C@_0BH@MPHCPCAM@java?1io?1FileDescriptor@ 00000001800098b0     IOUtil.obj
 0002:000008c8       ??_C@_06NCGDPKCC@handle@   00000001800098c8     IOUtil.obj
 0002:000008d0       ??_C@_0BC@PPBACNOJ@Read?1write?5failed@ 00000001800098d0     IOUtil.obj
 0002:000008e4       ??_C@_05GGAEIDGJ@Drain@    00000001800098e4     IOUtil.obj
 0002:000008f0       ??_C@_0CB@EANIAHBH@sun?1nio?1ch?1Iocp$CompletionStatu@ 00000001800098f0     Iocp.obj
 0002:00000914       ??_C@_05KKCIMGE@error@     0000000180009914     Iocp.obj
 0002:00000920       ??_C@_0BB@LMCKIICB@bytesTransferred@ 0000000180009920     Iocp.obj
 0002:00000938       ??_C@_0O@HHOLMKBG@completionKey@ 0000000180009938     Iocp.obj
 0002:00000948       ??_C@_0L@GFMJGGB@overlapped@ 0000000180009948     Iocp.obj
 0002:00000958       ??_C@_0BO@HNKCMKLP@CreateIoCompletionPort?5failed@ 0000000180009958     Iocp.obj
 0002:00000978       ??_C@_0CB@GOEOMHMA@GetQueuedCompletionStatus?5faile@ 0000000180009978     Iocp.obj
 0002:000009a0       ??_C@_0BL@IDOBBHMP@PostQueuedCompletionStatus@ 00000001800099a0     Iocp.obj
 0002:000009c0       ??_C@_0N@MNOMAIIN@Flush?5failed@ 00000001800099c0     MappedByteBuffer.obj
 0002:000009d0       ??_C@_06HBELJPBO@socket@   00000001800099d0     Net.obj
 0002:000009d8       ??_C@_0N@JOEJINBO@fastLoopback@ 00000001800099d8     Net.obj
 0002:000009e8       ??_C@_04NPNJNMMP@bind@     00000001800099e8     Net.obj
 0002:000009f0       ??_C@_06OODDLKLE@listen@   00000001800099f0     Net.obj
 0002:000009f8       ??_C@_07KAIBNCHO@connect@  00000001800099f8     Net.obj
 0002:00000a00       ??_C@_0M@ODFENJLC@getsockname@ 0000000180009a00     Net.obj
 0002:00000a10       ??_C@_08FIACBBDA@shutdown@ 0000000180009a10     Net.obj
 0002:00000a20       ??_C@_0O@BMGFIIHF@Accept?5failed@ 0000000180009a20     ServerSocketChannelImpl.obj
 0002:00000a30       ??_C@_0BF@LNJHKELF@java?1net?1InetAddress@ 0000000180009a30     SocketChannelImpl.obj
 0002:00000a48       ??_C@_07LHEPONKL@address@  0000000180009a48     SocketChannelImpl.obj
 0002:00000a50       ??_C@_0L@DEFCDCGF@getsockopt@ 0000000180009a50     SocketChannelImpl.obj
 0002:00000a60       ??_C@_0BD@MOAOKNAP@Vector?5read?5failed@ 0000000180009a60     SocketDispatcher.obj
 0002:00000a78       ??_C@_0BE@IPALPBFO@Vector?5write?5failed@ 0000000180009a78     SocketDispatcher.obj
 0002:00000a90       ??_C@_0BE@EFPANNNH@Socket?5close?5failed@ 0000000180009a90     SocketDispatcher.obj
 0002:00000aa8       ??_C@_0BA@KDJDNLHD@ReadFile?5failed@ 0000000180009aa8     WindowsAsynchronousFileChannelImpl.obj
 0002:00000ab8       ??_C@_0BB@IBAPLIEE@WriteFile?5failed@ 0000000180009ab8     WindowsAsynchronousFileChannelImpl.obj
 0002:00000ad0       ??_C@_0O@FPJGNADN@socket?5failed@ 0000000180009ad0     WindowsAsynchronousServerSocketChannelImpl.obj
 0002:00000ae0       ??_C@_0BA@PBEMOOLP@WSAIoctl?5failed@ 0000000180009ae0     WindowsAsynchronousServerSocketChannelImpl.obj
 0002:00000af0       ??_C@_0BA@CMPAPNB@AcceptEx?5failed@ 0000000180009af0     WindowsAsynchronousServerSocketChannelImpl.obj
 0002:00000b00       ??_C@_0BD@FFLNFFAC@closesocket?5failed@ 0000000180009b00     WindowsAsynchronousServerSocketChannelImpl.obj
 0002:00000b18       ??_C@_0BB@COIIDLME@ConnectEx?5failed@ 0000000180009b18     WindowsAsynchronousSocketChannelImpl.obj
 0002:00000b30       ??_C@_0BA@GMHHDNNI@shutdown?5failed@ 0000000180009b30     WindowsAsynchronousSocketChannelImpl.obj
 0002:00000b40       ??_C@_04PFANPMCN@?$CII?$CJV@ 0000000180009b40     WindowsNativeDispatcher.obj
 0002:00000b48       ??_C@_0BM@FOMEEEOI@sun?1nio?1fs?1WindowsException@ 0000000180009b48     WindowsNativeDispatcher.obj
 0002:00000b68       ??_C@_0CN@IAHHKCCP@sun?1nio?1fs?1WindowsNativeDispatc@ 0000000180009b68     WindowsNativeDispatcher.obj
 0002:00000b98       ??_C@_0BD@JFADHEFE@Ljava?1lang?1String?$DL@ 0000000180009b98     WindowsNativeDispatcher.obj
 0002:00000bac       ??_C@_04MEMAJGDJ@name@     0000000180009bac     WindowsNativeDispatcher.obj
 0002:00000bb8       ??_C@_0L@HNMJPKNA@attributes@ 0000000180009bb8     WindowsNativeDispatcher.obj
 0002:00000bc8       ??_C@_0CP@OGPMEFOM@sun?1nio?1fs?1WindowsNativeDispatc@ 0000000180009bc8     WindowsNativeDispatcher.obj
 0002:00000bf8       ??_C@_0DF@OBLOOIFM@sun?1nio?1fs?1WindowsNativeDispatc@ 0000000180009bf8     WindowsNativeDispatcher.obj
 0002:00000c30       ??_C@_0P@BFNHNOMJ@fileSystemName@ 0000000180009c30     WindowsNativeDispatcher.obj
 0002:00000c40       ??_C@_0L@HCGAGGAJ@volumeName@ 0000000180009c40     WindowsNativeDispatcher.obj
 0002:00000c50       ??_C@_0BD@ILMPNPNH@volumeSerialNumber@ 0000000180009c50     WindowsNativeDispatcher.obj
 0002:00000c64       ??_C@_05GECEPKB@flags@     0000000180009c64     WindowsNativeDispatcher.obj
 0002:00000c70       ??_C@_0DB@OGAJBKPO@sun?1nio?1fs?1WindowsNativeDispatc@ 0000000180009c70     WindowsNativeDispatcher.obj
 0002:00000ca8       ??_C@_0BD@LDNCHAFG@freeBytesAvailable@ 0000000180009ca8     WindowsNativeDispatcher.obj
 0002:00000cc0       ??_C@_0BD@FIEGHADN@totalNumberOfBytes@ 0000000180009cc0     WindowsNativeDispatcher.obj
 0002:00000cd8       ??_C@_0BH@DLDLDEPI@totalNumberOfFreeBytes@ 0000000180009cd8     WindowsNativeDispatcher.obj
 0002:00000cf0       ??_C@_0P@EEANGJCF@bytesPerSector@ 0000000180009cf0     WindowsNativeDispatcher.obj
 0002:00000d00       ??_C@_0CL@IEKIAJIE@sun?1nio?1fs?1WindowsNativeDispatc@ 0000000180009d00     WindowsNativeDispatcher.obj
 0002:00000d2c       ??_C@_06LKIIGAOE@domain@   0000000180009d2c     WindowsNativeDispatcher.obj
 0002:00000d34       ??_C@_03MMGHDJKG@use@      0000000180009d34     WindowsNativeDispatcher.obj
 0002:00000d38       ??_C@_0DC@CMOGENGN@sun?1nio?1fs?1WindowsNativeDispatc@ 0000000180009d38     WindowsNativeDispatcher.obj
 0002:00000d70       ??_C@_08BCFBCIIE@aceCount@ 0000000180009d70     WindowsNativeDispatcher.obj
 0002:00000d80       ??_C@_0DE@MGDINMHA@sun?1nio?1fs?1WindowsNativeDispatc@ 0000000180009d80     WindowsNativeDispatcher.obj
 0002:00000db8       ??_C@_0CC@NMODGIKH@Unable?5to?5allocate?5LUID?5structu@ 0000000180009db8     WindowsNativeDispatcher.obj
 0002:00000de0       ??_C@_0BI@COMCEALI@GetFullPathNameW?5failed@ 0000000180009de0     WindowsNativeDispatcher.obj
 0002:00000df8       ??_C@_0CB@DJOGFDBC@native?5memory?5allocation?5failur@ 0000000180009df8     WindowsNativeDispatcher.obj
 0002:00000e20       ??_C@_0CB@BLMDNHEM@GetFinalPathNameByHandleW?5faile@ 0000000180009e20     WindowsNativeDispatcher.obj
 0002:00000e48       _pDefaultRawDllMain        0000000180009e48     MSVCRT:dll_dllmain.obj
 0002:00000e48       _pRawDllMain               0000000180009e48     MSVCRT:dll_dllmain.obj
 0002:00000e60       __xmm@ffffffffffffffffffffffffffffffff 0000000180009e60     MSVCRT:utility.obj
 0002:00000e70       _load_config_used          0000000180009e70     MSVCRT:loadcfg.obj
 0002:00001080       __volatile_metadata        000000018000a080     <linker-defined>
 0002:000013a0       __rtc_iaa                  000000018000a3a0     MSVCRT:initsect.obj
 0002:000013a8       __rtc_izz                  000000018000a3a8     MSVCRT:initsect.obj
 0002:000013b0       __rtc_taa                  000000018000a3b0     MSVCRT:initsect.obj
 0002:000013b8       __rtc_tzz                  000000018000a3b8     MSVCRT:initsect.obj
 0002:00004340       __IMPORT_DESCRIPTOR_WS2_32 000000018000d340     ws2_32:WS2_32.dll
 0002:00004354       __IMPORT_DESCRIPTOR_java   000000018000d354     java:java.dll
 0002:00004368       __IMPORT_DESCRIPTOR_net    000000018000d368     net:net.dll
 0002:0000437c       __IMPORT_DESCRIPTOR_ADVAPI32 000000018000d37c     advapi32:ADVAPI32.dll
 0002:00004390       __IMPORT_DESCRIPTOR_MSWSOCK 000000018000d390     Mswsock:MSWSOCK.dll
 0002:000043a4       __IMPORT_DESCRIPTOR_KERNEL32 000000018000d3a4     kernel32:KERNEL32.dll
 0002:000043b8       __IMPORT_DESCRIPTOR_VCRUNTIME140 000000018000d3b8     vcruntime:VCRUNTIME140.dll
 0002:000043cc       __IMPORT_DESCRIPTOR_api-ms-win-crt-heap-l1-1-0 000000018000d3cc     ucrt:api-ms-win-crt-heap-l1-1-0.dll
 0002:000043e0       __IMPORT_DESCRIPTOR_api-ms-win-crt-stdio-l1-1-0 000000018000d3e0     ucrt:api-ms-win-crt-stdio-l1-1-0.dll
 0002:000043f4       __IMPORT_DESCRIPTOR_api-ms-win-crt-string-l1-1-0 000000018000d3f4     ucrt:api-ms-win-crt-string-l1-1-0.dll
 0002:00004408       __IMPORT_DESCRIPTOR_api-ms-win-crt-runtime-l1-1-0 000000018000d408     ucrt:api-ms-win-crt-runtime-l1-1-0.dll
 0002:0000441c       __NULL_IMPORT_DESCRIPTOR   000000018000d41c     ws2_32:WS2_32.dll
 0003:00000010       __security_cookie_complement 000000018000f010     MSVCRT:gs_cookie.obj
 0003:00000018       __security_cookie          000000018000f018     MSVCRT:gs_cookie.obj
 0003:00000020       __scrt_native_dllmain_reason 000000018000f020     MSVCRT:utility.obj
 0003:00000028       __isa_available            000000018000f028     MSVCRT:cpu_disp.obj
 0003:0000002c       __isa_enabled              000000018000f02c     MSVCRT:cpu_disp.obj
 0003:00000030       __memset_fast_string_threshold 000000018000f030     MSVCRT:cpu_disp.obj
 0003:00000038       __memset_nt_threshold      000000018000f038     MSVCRT:cpu_disp.obj
 0003:00000040       __scrt_ucrt_dll_is_in_use  000000018000f040     MSVCRT:ucrt_stubs.obj
 0003:00000720       ?__type_info_root_node@@3U__type_info_node@@A 000000018000f720     MSVCRT:tncleanup.obj
 0003:00000730       ?_OptionsStorage@?1??__local_stdio_printf_options@@9@4_KA 000000018000f730     MSVCRT:default_local_stdio_options.obj
 0003:00000738       ?_OptionsStorage@?1??__local_stdio_scanf_options@@9@4_KA 000000018000f738     MSVCRT:default_local_stdio_options.obj
 0003:00000740       __scrt_current_native_startup_state 000000018000f740     MSVCRT:utility.obj
 0003:00000748       __scrt_native_startup_lock 000000018000f748     MSVCRT:utility.obj
 0003:00000788       __scrt_debugger_hook_flag  000000018000f788     MSVCRT:utility_desktop.obj
 0003:0000078c       __favor                    000000018000f78c     MSVCRT:cpu_disp.obj
 0003:00000790       __dyn_tls_init_callback    000000018000f790     <common>

 entry point at        0001:00006550

 Static symbols

 0000:fffed000       .debug$S                   0000000180000000     nio.exp
 0000:fffed000       .debug$S                   0000000180000000     vcruntime:VCRUNTIME140.dll
 0000:fffed000       .debug$S                   0000000180000000     vcruntime:VCRUNTIME140.dll
 0000:fffed000       .debug$S                   0000000180000000     vcruntime:VCRUNTIME140.dll
 0000:fffed000       .debug$S                   0000000180000000     vcruntime:VCRUNTIME140.dll
 0000:fffed000       .debug$S                   0000000180000000     vcruntime:VCRUNTIME140.dll
 0000:fffed000       .debug$S                   0000000180000000     vcruntime:VCRUNTIME140.dll
 0000:fffed000       .debug$S                   0000000180000000     ucrt:api-ms-win-crt-heap-l1-1-0.dll
 0000:fffed000       .debug$S                   0000000180000000     ucrt:api-ms-win-crt-heap-l1-1-0.dll
 0000:fffed000       .debug$S                   0000000180000000     ucrt:api-ms-win-crt-runtime-l1-1-0.dll
 0000:fffed000       .debug$S                   0000000180000000     ucrt:api-ms-win-crt-runtime-l1-1-0.dll
 0000:fffed000       .debug$S                   0000000180000000     ucrt:api-ms-win-crt-runtime-l1-1-0.dll
 0000:fffed000       .debug$S                   0000000180000000     ucrt:api-ms-win-crt-runtime-l1-1-0.dll
 0000:fffed000       .debug$S                   0000000180000000     ucrt:api-ms-win-crt-runtime-l1-1-0.dll
 0000:fffed000       .debug$S                   0000000180000000     ucrt:api-ms-win-crt-runtime-l1-1-0.dll
 0000:fffed000       .debug$S                   0000000180000000     ucrt:api-ms-win-crt-runtime-l1-1-0.dll
 0000:fffed000       .debug$S                   0000000180000000     ucrt:api-ms-win-crt-runtime-l1-1-0.dll
 0000:fffed000       .debug$S                   0000000180000000     ucrt:api-ms-win-crt-runtime-l1-1-0.dll
 0000:fffed000       .debug$S                   0000000180000000     ucrt:api-ms-win-crt-runtime-l1-1-0.dll
 0000:fffed000       .debug$S                   0000000180000000     ucrt:api-ms-win-crt-runtime-l1-1-0.dll
 0000:fffed000       .debug$S                   0000000180000000     ucrt:api-ms-win-crt-runtime-l1-1-0.dll
 0000:fffed000       .debug$S                   0000000180000000     ucrt:api-ms-win-crt-runtime-l1-1-0.dll
 0000:fffed000       .debug$S                   0000000180000000     ucrt:api-ms-win-crt-stdio-l1-1-0.dll
 0000:fffed000       .debug$S                   0000000180000000     ucrt:api-ms-win-crt-string-l1-1-0.dll
 0000:fffed000       .debug$S                   0000000180000000     Mswsock:MSWSOCK.dll
 0000:fffed000       .debug$S                   0000000180000000     advapi32:ADVAPI32.dll
 0000:fffed000       .debug$S                   0000000180000000     advapi32:ADVAPI32.dll
 0000:fffed000       .debug$S                   0000000180000000     advapi32:ADVAPI32.dll
 0000:fffed000       .debug$S                   0000000180000000     advapi32:ADVAPI32.dll
 0000:fffed000       .debug$S                   0000000180000000     advapi32:ADVAPI32.dll
 0000:fffed000       .debug$S                   0000000180000000     advapi32:ADVAPI32.dll
 0000:fffed000       .debug$S                   0000000180000000     advapi32:ADVAPI32.dll
 0000:fffed000       .debug$S                   0000000180000000     advapi32:ADVAPI32.dll
 0000:fffed000       .debug$S                   0000000180000000     advapi32:ADVAPI32.dll
 0000:fffed000       .debug$S                   0000000180000000     advapi32:ADVAPI32.dll
 0000:fffed000       .debug$S                   0000000180000000     advapi32:ADVAPI32.dll
 0000:fffed000       .debug$S                   0000000180000000     advapi32:ADVAPI32.dll
 0000:fffed000       .debug$S                   0000000180000000     advapi32:ADVAPI32.dll
 0000:fffed000       .debug$S                   0000000180000000     advapi32:ADVAPI32.dll
 0000:fffed000       .debug$S                   0000000180000000     advapi32:ADVAPI32.dll
 0000:fffed000       .debug$S                   0000000180000000     advapi32:ADVAPI32.dll
 0000:fffed000       .debug$S                   0000000180000000     advapi32:ADVAPI32.dll
 0000:fffed000       .debug$S                   0000000180000000     advapi32:ADVAPI32.dll
 0000:fffed000       .debug$S                   0000000180000000     advapi32:ADVAPI32.dll
 0000:fffed000       .debug$S                   0000000180000000     advapi32:ADVAPI32.dll
 0000:fffed000       .debug$S                   0000000180000000     advapi32:ADVAPI32.dll
 0000:fffed000       .debug$S                   0000000180000000     advapi32:ADVAPI32.dll
 0000:fffed000       .debug$S                   0000000180000000     advapi32:ADVAPI32.dll
 0000:fffed000       .debug$S                   0000000180000000     advapi32:ADVAPI32.dll
 0000:fffed000       .debug$S                   0000000180000000     advapi32:ADVAPI32.dll
 0000:fffed000       .debug$S                   0000000180000000     advapi32:ADVAPI32.dll
 0000:fffed000       .debug$S                   0000000180000000     advapi32:ADVAPI32.dll
 0000:fffed000       .debug$S                   0000000180000000     advapi32:ADVAPI32.dll
 0000:fffed000       .debug$S                   0000000180000000     advapi32:ADVAPI32.dll
 0000:fffed000       .debug$S                   0000000180000000     kernel32:KERNEL32.dll
 0000:fffed000       .debug$S                   0000000180000000     kernel32:KERNEL32.dll
 0000:fffed000       .debug$S                   0000000180000000     kernel32:KERNEL32.dll
 0000:fffed000       .debug$S                   0000000180000000     kernel32:KERNEL32.dll
 0000:fffed000       .debug$S                   0000000180000000     kernel32:KERNEL32.dll
 0000:fffed000       .debug$S                   0000000180000000     kernel32:KERNEL32.dll
 0000:fffed000       .debug$S                   0000000180000000     kernel32:KERNEL32.dll
 0000:fffed000       .debug$S                   0000000180000000     kernel32:KERNEL32.dll
 0000:fffed000       .debug$S                   0000000180000000     kernel32:KERNEL32.dll
 0000:fffed000       .debug$S                   0000000180000000     kernel32:KERNEL32.dll
 0000:fffed000       .debug$S                   0000000180000000     kernel32:KERNEL32.dll
 0000:fffed000       .debug$S                   0000000180000000     kernel32:KERNEL32.dll
 0000:fffed000       .debug$S                   0000000180000000     kernel32:KERNEL32.dll
 0000:fffed000       .debug$S                   0000000180000000     kernel32:KERNEL32.dll
 0000:fffed000       .debug$S                   0000000180000000     kernel32:KERNEL32.dll
 0000:fffed000       .debug$S                   0000000180000000     kernel32:KERNEL32.dll
 0000:fffed000       .debug$S                   0000000180000000     kernel32:KERNEL32.dll
 0000:fffed000       .debug$S                   0000000180000000     kernel32:KERNEL32.dll
 0000:fffed000       .debug$S                   0000000180000000     kernel32:KERNEL32.dll
 0000:fffed000       .debug$S                   0000000180000000     kernel32:KERNEL32.dll
 0000:fffed000       .debug$S                   0000000180000000     kernel32:KERNEL32.dll
 0000:fffed000       .debug$S                   0000000180000000     kernel32:KERNEL32.dll
 0000:fffed000       .debug$S                   0000000180000000     kernel32:KERNEL32.dll
 0000:fffed000       .debug$S                   0000000180000000     kernel32:KERNEL32.dll
 0000:fffed000       .debug$S                   0000000180000000     kernel32:KERNEL32.dll
 0000:fffed000       .debug$S                   0000000180000000     kernel32:KERNEL32.dll
 0000:fffed000       .debug$S                   0000000180000000     kernel32:KERNEL32.dll
 0000:fffed000       .debug$S                   0000000180000000     kernel32:KERNEL32.dll
 0000:fffed000       .debug$S                   0000000180000000     kernel32:KERNEL32.dll
 0000:fffed000       .debug$S                   0000000180000000     kernel32:KERNEL32.dll
 0000:fffed000       .debug$S                   0000000180000000     kernel32:KERNEL32.dll
 0000:fffed000       .debug$S                   0000000180000000     kernel32:KERNEL32.dll
 0000:fffed000       .debug$S                   0000000180000000     kernel32:KERNEL32.dll
 0000:fffed000       .debug$S                   0000000180000000     kernel32:KERNEL32.dll
 0000:fffed000       .debug$S                   0000000180000000     kernel32:KERNEL32.dll
 0000:fffed000       .debug$S                   0000000180000000     kernel32:KERNEL32.dll
 0000:fffed000       .debug$S                   0000000180000000     kernel32:KERNEL32.dll
 0000:fffed000       .debug$S                   0000000180000000     kernel32:KERNEL32.dll
 0000:fffed000       .debug$S                   0000000180000000     kernel32:KERNEL32.dll
 0000:fffed000       .debug$S                   0000000180000000     kernel32:KERNEL32.dll
 0000:fffed000       .debug$S                   0000000180000000     kernel32:KERNEL32.dll
 0000:fffed000       .debug$S                   0000000180000000     kernel32:KERNEL32.dll
 0000:fffed000       .debug$S                   0000000180000000     kernel32:KERNEL32.dll
 0000:fffed000       .debug$S                   0000000180000000     kernel32:KERNEL32.dll
 0000:fffed000       .debug$S                   0000000180000000     kernel32:KERNEL32.dll
 0000:fffed000       .debug$S                   0000000180000000     kernel32:KERNEL32.dll
 0000:fffed000       .debug$S                   0000000180000000     kernel32:KERNEL32.dll
 0000:fffed000       .debug$S                   0000000180000000     kernel32:KERNEL32.dll
 0000:fffed000       .debug$S                   0000000180000000     kernel32:KERNEL32.dll
 0000:fffed000       .debug$S                   0000000180000000     kernel32:KERNEL32.dll
 0000:fffed000       .debug$S                   0000000180000000     kernel32:KERNEL32.dll
 0000:fffed000       .debug$S                   0000000180000000     kernel32:KERNEL32.dll
 0000:fffed000       .debug$S                   0000000180000000     kernel32:KERNEL32.dll
 0000:fffed000       .debug$S                   0000000180000000     kernel32:KERNEL32.dll
 0000:fffed000       .debug$S                   0000000180000000     kernel32:KERNEL32.dll
 0000:fffed000       .debug$S                   0000000180000000     kernel32:KERNEL32.dll
 0000:fffed000       .debug$S                   0000000180000000     kernel32:KERNEL32.dll
 0000:fffed000       .debug$S                   0000000180000000     kernel32:KERNEL32.dll
 0000:fffed000       .debug$S                   0000000180000000     kernel32:KERNEL32.dll
 0000:fffed000       .debug$S                   0000000180000000     kernel32:KERNEL32.dll
 0000:fffed000       .debug$S                   0000000180000000     kernel32:KERNEL32.dll
 0000:fffed000       .debug$S                   0000000180000000     kernel32:KERNEL32.dll
 0000:fffed000       .debug$S                   0000000180000000     kernel32:KERNEL32.dll
 0000:fffed000       .debug$S                   0000000180000000     kernel32:KERNEL32.dll
 0000:fffed000       .debug$S                   0000000180000000     kernel32:KERNEL32.dll
 0000:fffed000       .debug$S                   0000000180000000     kernel32:KERNEL32.dll
 0000:fffed000       .debug$S                   0000000180000000     kernel32:KERNEL32.dll
 0000:fffed000       .debug$S                   0000000180000000     kernel32:KERNEL32.dll
 0000:fffed000       .debug$S                   0000000180000000     kernel32:KERNEL32.dll
 0000:fffed000       .debug$S                   0000000180000000     kernel32:KERNEL32.dll
 0000:fffed000       .debug$S                   0000000180000000     kernel32:KERNEL32.dll
 0000:fffed000       .debug$S                   0000000180000000     kernel32:KERNEL32.dll
 0000:fffed000       .debug$S                   0000000180000000     kernel32:KERNEL32.dll
 0000:fffed000       .debug$S                   0000000180000000     kernel32:KERNEL32.dll
 0000:fffed000       .debug$S                   0000000180000000     ws2_32:WS2_32.dll
 0000:fffed000       .debug$S                   0000000180000000     ws2_32:WS2_32.dll
 0000:fffed000       .debug$S                   0000000180000000     ws2_32:WS2_32.dll
 0000:fffed000       .debug$S                   0000000180000000     ws2_32:WS2_32.dll
 0000:fffed000       .debug$S                   0000000180000000     ws2_32:WS2_32.dll
 0000:fffed000       .debug$S                   0000000180000000     ws2_32:WS2_32.dll
 0000:fffed000       .debug$S                   0000000180000000     ws2_32:WS2_32.dll
 0000:fffed000       .debug$S                   0000000180000000     ws2_32:WS2_32.dll
 0000:fffed000       .debug$S                   0000000180000000     ws2_32:WS2_32.dll
 0000:fffed000       .debug$S                   0000000180000000     ws2_32:WS2_32.dll
 0000:fffed000       .debug$S                   0000000180000000     ws2_32:WS2_32.dll
 0000:fffed000       .debug$S                   0000000180000000     ws2_32:WS2_32.dll
 0000:fffed000       .debug$S                   0000000180000000     ws2_32:WS2_32.dll
 0000:fffed000       .debug$S                   0000000180000000     ws2_32:WS2_32.dll
 0000:fffed000       .debug$S                   0000000180000000     ws2_32:WS2_32.dll
 0000:fffed000       .debug$S                   0000000180000000     ws2_32:WS2_32.dll
 0000:fffed000       .debug$S                   0000000180000000     ws2_32:WS2_32.dll
 0000:fffed000       .debug$S                   0000000180000000     ws2_32:WS2_32.dll
 0000:fffed000       .debug$S                   0000000180000000     ws2_32:WS2_32.dll
 0000:fffed000       .debug$S                   0000000180000000     ws2_32:WS2_32.dll
 0000:fffed000       .debug$S                   0000000180000000     ws2_32:WS2_32.dll
 0000:fffed000       .debug$S                   0000000180000000     ws2_32:WS2_32.dll
 0000:fffed000       .debug$S                   0000000180000000     ws2_32:WS2_32.dll
 0000:fffed000       .debug$S                   0000000180000000     ws2_32:WS2_32.dll
 0000:fffed000       .debug$S                   0000000180000000     java:java.dll
 0000:fffed000       .debug$S                   0000000180000000     java:java.dll
 0000:fffed000       .debug$S                   0000000180000000     java:java.dll
 0000:fffed000       .debug$S                   0000000180000000     java:java.dll
 0000:fffed000       .debug$S                   0000000180000000     java:java.dll
 0000:fffed000       .debug$S                   0000000180000000     java:java.dll
 0000:fffed000       .debug$S                   0000000180000000     net:net.dll
 0000:fffed000       .debug$S                   0000000180000000     net:net.dll
 0000:fffed000       .debug$S                   0000000180000000     net:net.dll
 0000:fffed000       .debug$S                   0000000180000000     net:net.dll
 0000:fffed000       .debug$S                   0000000180000000     net:net.dll
 0000:fffed000       .debug$S                   0000000180000000     net:net.dll
 0000:fffed000       .debug$S                   0000000180000000     net:net.dll
 0000:fffed000       .debug$S                   0000000180000000     net:net.dll
 0000:fffed000       .debug$S                   0000000180000000     net:net.dll
 0000:fffed000       .debug$S                   0000000180000000     net:net.dll
 0000:fffed000       .debug$S                   0000000180000000     net:net.dll
 0000:fffed000       .debug$S                   0000000180000000     net:net.dll
 0001:00002ca0       setGroupSourceReqOption    0000000180003ca0 f   Net.obj
 0001:00005b30       throwWindowsException      0000000180006b30 f   WindowsNativeDispatcher.obj
 0001:000061a0       $$000000                   00000001800071a0     MSVCRT:amdsecgs.obj
 0001:000061d0       $$000000                   00000001800071d0     MSVCRT:chkstk.obj
 0001:00006230       ?dllmain_crt_dispatch@@YAHQEAUHINSTANCE__@@KQEAX@Z 0000000180007230 f   MSVCRT:dll_dllmain.obj
 0001:00006280       ?dllmain_crt_process_attach@@YAHQEAUHINSTANCE__@@QEAX@Z 0000000180007280 f   MSVCRT:dll_dllmain.obj
 0001:00006398       ?dllmain_crt_process_detach@@YAH_N@Z 0000000180007398 f   MSVCRT:dll_dllmain.obj
 0001:0000641c       ?dllmain_dispatch@@YAHQEAUHINSTANCE__@@KQEAX@Z 000000018000741c f   MSVCRT:dll_dllmain.obj
 0001:00006698       capture_previous_context   0000000180007698 f   MSVCRT:gs_report.obj
 0001:00006f40       $$000000                   0000000180007f40     MSVCRT:guard_dispatch.obj
 0001:00006f60       $$000000                   0000000180007f60     MSVCRT:guard_xfg_dispatch.obj
 0001:00006f76       ?fin$0@?0??dllmain_crt_process_attach@@YAHQEAUHINSTANCE__@@QEAX@Z@4HA 0000000180007f76 f   MSVCRT:dll_dllmain.obj
 0001:00006f8d       ?fin$0@?0??dllmain_crt_process_detach@@YAH_N@Z@4HA 0000000180007f8d f   MSVCRT:dll_dllmain.obj
 0001:00006fa6       ?fin$1@?0??dllmain_crt_process_detach@@YAH_N@Z@4HA 0000000180007fa6 f   MSVCRT:dll_dllmain.obj
 0001:00006fba       ?filt$0@?0??dllmain_dispatch@@YAHQEAUHINSTANCE__@@KQEAX@Z@4HA 0000000180007fba f   MSVCRT:dll_dllmain.obj
 0001:00006ff0       __scrt_is_nonwritable_in_current_image$filt$0 0000000180007ff0 f   MSVCRT:utility.obj
 0002:00000e50       GS_ExceptionPointers       0000000180009e50     MSVCRT:gs_report.obj
 0002:000013c0       $unwind$Java_sun_nio_ch_DatagramChannelImpl_initIDs 000000018000a3c0     DatagramChannelImpl.obj
 0002:000013c0       $unwind$Java_sun_nio_ch_FileDispatcherImpl_seek0 000000018000a3c0     FileDispatcherImpl.obj
 0002:000013c0       $unwind$Java_sun_nio_ch_FileDispatcherImpl_truncate0 000000018000a3c0     FileDispatcherImpl.obj
 0002:000013c0       $unwind$Java_sun_nio_ch_FileKey_initIDs 000000018000a3c0     FileKey.obj
 0002:000013c0       $unwind$Java_sun_nio_ch_IOUtil_initIDs 000000018000a3c0     IOUtil.obj
 0002:000013c0       $unwind$Java_sun_nio_ch_Iocp_createIoCompletionPort 000000018000a3c0     Iocp.obj
 0002:000013c0       $unwind$Java_sun_nio_ch_Iocp_initIDs 000000018000a3c0     Iocp.obj
 0002:000013c0       $unwind$Java_sun_nio_ch_Net_listen 000000018000a3c0     Net.obj
 0002:000013c0       $unwind$Java_sun_nio_ch_Net_shutdown 000000018000a3c0     Net.obj
 0002:000013c0       $unwind$Java_sun_nio_ch_ServerSocketChannelImpl_initIDs 000000018000a3c0     ServerSocketChannelImpl.obj
 0002:000013c0       $unwind$Java_sun_nio_ch_ServerSocketChannelImpl_listen 000000018000a3c0     ServerSocketChannelImpl.obj
 0002:000013c0       $unwind$Java_sun_nio_fs_WindowsNativeDispatcher_ConvertSidToStringSid 000000018000a3c0     WindowsNativeDispatcher.obj
 0002:000013c0       $unwind$Java_sun_nio_fs_WindowsNativeDispatcher_CreateEvent 000000018000a3c0     WindowsNativeDispatcher.obj
 0002:000013c0       $unwind$Java_sun_nio_fs_WindowsNativeDispatcher_CreateIoCompletionPort 000000018000a3c0     WindowsNativeDispatcher.obj
 0002:000013c0       $unwind$Java_sun_nio_fs_WindowsNativeDispatcher_FindFirstFile1 000000018000a3c0     WindowsNativeDispatcher.obj
 0002:000013c0       $unwind$Java_sun_nio_fs_WindowsNativeDispatcher_GetFileAttributes0 000000018000a3c0     WindowsNativeDispatcher.obj
 0002:000013c0       $unwind$Java_sun_nio_fs_WindowsNativeDispatcher_GetLogicalDrives 000000018000a3c0     WindowsNativeDispatcher.obj
 0002:000013c0       $unwind$_RTC_Initialize    000000018000a3c0     MSVCRT:initsect.obj
 0002:000013c0       $unwind$_RTC_Terminate     000000018000a3c0     MSVCRT:initsect.obj
 0002:000013cc       $unwind$Java_sun_nio_ch_DatagramChannelImpl_disconnect0 000000018000a3cc     DatagramChannelImpl.obj
 0002:000013e0       $unwind$Java_sun_nio_ch_DatagramChannelImpl_receive0 000000018000a3e0     DatagramChannelImpl.obj
 0002:000013fc       $unwind$Java_sun_nio_ch_DatagramChannelImpl_send0 000000018000a3fc     DatagramChannelImpl.obj
 0002:00001414       $unwind$purgeOutstandingICMP 000000018000a414     DatagramChannelImpl.obj
 0002:00001434       $unwind$Java_sun_nio_ch_DatagramDispatcher_read0 000000018000a434     DatagramDispatcher.obj
 0002:00001448       $unwind$Java_sun_nio_ch_DatagramDispatcher_readv0 000000018000a448     DatagramDispatcher.obj
 0002:00001448       $unwind$Java_sun_nio_ch_SocketDispatcher_readv0 000000018000a448     SocketDispatcher.obj
 0002:00001460       $unwind$Java_sun_nio_ch_DatagramDispatcher_write0 000000018000a460     DatagramDispatcher.obj
 0002:00001474       $unwind$Java_sun_nio_ch_DatagramDispatcher_writev0 000000018000a474     DatagramDispatcher.obj
 0002:0000148c       $unwind$Java_sun_nio_ch_FileChannelImpl_map0 000000018000a48c     FileChannelImpl.obj
 0002:000014a8       $unwind$Java_sun_nio_ch_FileChannelImpl_unmap0 000000018000a4a8     FileChannelImpl.obj
 0002:000014a8       $unwind$Java_sun_nio_ch_FileDispatcherImpl_close0 000000018000a4a8     FileDispatcherImpl.obj
 0002:000014a8       $unwind$Java_sun_nio_ch_FileDispatcherImpl_force0 000000018000a4a8     FileDispatcherImpl.obj
 0002:000014a8       $unwind$Java_sun_nio_ch_FileDispatcherImpl_size0 000000018000a4a8     FileDispatcherImpl.obj
 0002:000014a8       $unwind$Java_sun_nio_ch_Iocp_postQueuedCompletionStatus 000000018000a4a8     Iocp.obj
 0002:000014a8       $unwind$Java_sun_nio_ch_SocketChannelImpl_initIDs 000000018000a4a8     SocketChannelImpl.obj
 0002:000014a8       $unwind$Java_sun_nio_ch_SocketDispatcher_close0 000000018000a4a8     SocketDispatcher.obj
 0002:000014a8       $unwind$Java_sun_nio_ch_WindowsAsynchronousServerSocketChannelImpl_closesocket0 000000018000a4a8     WindowsAsynchronousServerSocketChannelImpl.obj
 0002:000014a8       $unwind$Java_sun_nio_ch_WindowsAsynchronousSocketChannelImpl_closesocket0 000000018000a4a8     WindowsAsynchronousSocketChannelImpl.obj
 0002:000014a8       $unwind$Java_sun_nio_ch_WindowsAsynchronousSocketChannelImpl_shutdown0 000000018000a4a8     WindowsAsynchronousSocketChannelImpl.obj
 0002:000014a8       $unwind$Java_sun_nio_fs_WindowsNativeDispatcher_CancelIo 000000018000a4a8     WindowsNativeDispatcher.obj
 0002:000014a8       $unwind$Java_sun_nio_fs_WindowsNativeDispatcher_ConvertStringSidToSid0 000000018000a4a8     WindowsNativeDispatcher.obj
 0002:000014a8       $unwind$Java_sun_nio_fs_WindowsNativeDispatcher_CreateHardLink0 000000018000a4a8     WindowsNativeDispatcher.obj
 0002:000014a8       $unwind$Java_sun_nio_fs_WindowsNativeDispatcher_CreateSymbolicLink0 000000018000a4a8     WindowsNativeDispatcher.obj
 0002:000014a8       $unwind$Java_sun_nio_fs_WindowsNativeDispatcher_DeleteFile0 000000018000a4a8     WindowsNativeDispatcher.obj
 0002:000014a8       $unwind$Java_sun_nio_fs_WindowsNativeDispatcher_FindClose 000000018000a4a8     WindowsNativeDispatcher.obj
 0002:000014a8       $unwind$Java_sun_nio_fs_WindowsNativeDispatcher_GetAce 000000018000a4a8     WindowsNativeDispatcher.obj
 0002:000014a8       $unwind$Java_sun_nio_fs_WindowsNativeDispatcher_GetFileAttributesEx0 000000018000a4a8     WindowsNativeDispatcher.obj
 0002:000014a8       $unwind$Java_sun_nio_fs_WindowsNativeDispatcher_GetFileInformationByHandle 000000018000a4a8     WindowsNativeDispatcher.obj
 0002:000014a8       $unwind$Java_sun_nio_fs_WindowsNativeDispatcher_GetSecurityDescriptorOwner 000000018000a4a8     WindowsNativeDispatcher.obj
 0002:000014a8       $unwind$Java_sun_nio_fs_WindowsNativeDispatcher_InitializeAcl 000000018000a4a8     WindowsNativeDispatcher.obj
 0002:000014a8       $unwind$Java_sun_nio_fs_WindowsNativeDispatcher_InitializeSecurityDescriptor 000000018000a4a8     WindowsNativeDispatcher.obj
 0002:000014a8       $unwind$Java_sun_nio_fs_WindowsNativeDispatcher_MoveFileEx0 000000018000a4a8     WindowsNativeDispatcher.obj
 0002:000014a8       $unwind$Java_sun_nio_fs_WindowsNativeDispatcher_OpenProcessToken 000000018000a4a8     WindowsNativeDispatcher.obj
 0002:000014a8       $unwind$Java_sun_nio_fs_WindowsNativeDispatcher_OpenThreadToken 000000018000a4a8     WindowsNativeDispatcher.obj
 0002:000014a8       $unwind$Java_sun_nio_fs_WindowsNativeDispatcher_PostQueuedCompletionStatus 000000018000a4a8     WindowsNativeDispatcher.obj
 0002:000014a8       $unwind$Java_sun_nio_fs_WindowsNativeDispatcher_RemoveDirectory0 000000018000a4a8     WindowsNativeDispatcher.obj
 0002:000014a8       $unwind$Java_sun_nio_fs_WindowsNativeDispatcher_SetEndOfFile 000000018000a4a8     WindowsNativeDispatcher.obj
 0002:000014a8       $unwind$Java_sun_nio_fs_WindowsNativeDispatcher_SetFileAttributes0 000000018000a4a8     WindowsNativeDispatcher.obj
 0002:000014a8       $unwind$Java_sun_nio_fs_WindowsNativeDispatcher_SetFileSecurity0 000000018000a4a8     WindowsNativeDispatcher.obj
 0002:000014a8       $unwind$Java_sun_nio_fs_WindowsNativeDispatcher_SetSecurityDescriptorDacl 000000018000a4a8     WindowsNativeDispatcher.obj
 0002:000014a8       $unwind$Java_sun_nio_fs_WindowsNativeDispatcher_SetSecurityDescriptorOwner 000000018000a4a8     WindowsNativeDispatcher.obj
 0002:000014a8       $unwind$Java_sun_nio_fs_WindowsNativeDispatcher_SetThreadToken 000000018000a4a8     WindowsNativeDispatcher.obj
 0002:000014a8       $unwind$throwWindowsException 000000018000a4a8     WindowsNativeDispatcher.obj
 0002:000014a8       $unwind$__raise_securityfailure 000000018000a4a8     MSVCRT:gs_report.obj
 0002:000014a8       $unwind$__scrt_initialize_crt 000000018000a4a8     MSVCRT:utility.obj
 0002:000014a8       $unwind$__scrt_initialize_onexit_tables 000000018000a4a8     MSVCRT:utility.obj
 0002:000014a8       $unwind$__scrt_release_startup_lock 000000018000a4a8     MSVCRT:utility.obj
 0002:000014a8       $unwind$__scrt_uninitialize_crt 000000018000a4a8     MSVCRT:utility.obj
 0002:000014b0       $unwind$Java_sun_nio_ch_FileChannelImpl_transferTo0 000000018000a4b0     FileChannelImpl.obj
 0002:000014c4       $unwind$Java_sun_nio_ch_FileChannelImpl_initIDs 000000018000a4c4     FileChannelImpl.obj
 0002:000014c4       $unwind$Java_sun_nio_ch_FileDispatcherImpl_lock0 000000018000a4c4     FileDispatcherImpl.obj
 0002:000014c4       $unwind$Java_sun_nio_ch_FileDispatcherImpl_release0 000000018000a4c4     FileDispatcherImpl.obj
 0002:000014d4       $unwind$Java_sun_nio_ch_FileDispatcherImpl_duplicateHandle 000000018000a4d4     FileDispatcherImpl.obj
 0002:000014d4       $unwind$Java_sun_nio_ch_FileDispatcherImpl_read0 000000018000a4d4     FileDispatcherImpl.obj
 0002:000014d4       $unwind$Java_sun_nio_ch_Net_setInterface4 000000018000a4d4     Net.obj
 0002:000014e0       $unwind$Java_sun_nio_ch_FileDispatcherImpl_pread0 000000018000a4e0     FileDispatcherImpl.obj
 0002:000014e0       $unwind$Java_sun_nio_ch_FileDispatcherImpl_pwrite0 000000018000a4e0     FileDispatcherImpl.obj
 0002:000014e0       $unwind$Java_sun_nio_ch_FileDispatcherImpl_write0 000000018000a4e0     FileDispatcherImpl.obj
 0002:000014f0       $unwind$Java_sun_nio_ch_FileDispatcherImpl_readv0 000000018000a4f0     FileDispatcherImpl.obj
 0002:00001508       $unwind$Java_sun_nio_ch_FileDispatcherImpl_writev0 000000018000a508     FileDispatcherImpl.obj
 0002:00001524       $unwind$Java_sun_nio_ch_FileDispatcherImpl_setDirect0 000000018000a524     FileDispatcherImpl.obj
 0002:00001534       $unwind$Java_sun_nio_ch_FileKey_init 000000018000a534     FileKey.obj
 0002:00001548       $unwind$convertLongReturnVal 000000018000a548     IOUtil.obj
 0002:00001548       $unwind$convertReturnVal   000000018000a548     IOUtil.obj
 0002:00001548       $unwind$Java_sun_nio_ch_Net_isIPv6Available0 000000018000a548     Net.obj
 0002:00001548       $unwind$handleSocketError  000000018000a548     SocketChannelImpl.obj
 0002:00001548       $unwind$Java_sun_nio_ch_WindowsSelectorImpl_setWakeupSocket0 000000018000a548     WindowsSelectorImpl.obj
 0002:00001548       $unwind$JNI_OnLoad         000000018000a548     nio_util.obj
 0002:00001548       $unwind$__scrt_initialize_default_local_stdio_options 000000018000a548     MSVCRT:default_local_stdio_options.obj
 0002:00001548       $unwind$?dllmain_crt_dispatch@@YAHQEAUHINSTANCE__@@KQEAX@Z 000000018000a548     MSVCRT:dll_dllmain.obj
 0002:00001548       $unwind$DllMain            000000018000a548     MSVCRT:dll_dllmain_stub.obj
 0002:00001548       $unwind$__GSHandlerCheck   000000018000a548     MSVCRT:gshandler.obj
 0002:00001548       $unwind$__scrt_acquire_startup_lock 000000018000a548     MSVCRT:utility.obj
 0002:00001548       $unwind$__scrt_dllmain_after_initialize_c 000000018000a548     MSVCRT:utility.obj
 0002:00001548       $unwind$__scrt_dllmain_before_initialize_c 000000018000a548     MSVCRT:utility.obj
 0002:00001548       $unwind$__scrt_dllmain_crt_thread_attach 000000018000a548     MSVCRT:utility.obj
 0002:00001548       $unwind$__scrt_dllmain_crt_thread_detach 000000018000a548     MSVCRT:utility.obj
 0002:00001548       $unwind$__scrt_dllmain_uninitialize_c 000000018000a548     MSVCRT:utility.obj
 0002:00001548       $unwind$__scrt_dllmain_uninitialize_critical 000000018000a548     MSVCRT:utility.obj
 0002:00001550       $unwind$Java_sun_nio_ch_IOUtil_drain 000000018000a550     IOUtil.obj
 0002:0000156c       $unwind$Java_sun_nio_ch_IOUtil_configureBlocking 000000018000a56c     IOUtil.obj
 0002:0000156c       $unwind$Java_sun_nio_fs_WindowsNativeDispatcher_FindNextFile 000000018000a56c     WindowsNativeDispatcher.obj
 0002:0000156c       $unwind$Java_sun_nio_fs_WindowsNativeDispatcher_LookupPrivilegeValue0 000000018000a56c     WindowsNativeDispatcher.obj
 0002:0000156c       $unwind$_DllMainCRTStartup 000000018000a56c     MSVCRT:dll_dllmain.obj
 0002:0000157c       $unwind$Java_sun_nio_ch_Iocp_getQueuedCompletionStatus 000000018000a57c     Iocp.obj
 0002:0000157c       $unwind$Java_sun_nio_fs_WindowsNativeDispatcher_GetQueuedCompletionStatus0 000000018000a57c     WindowsNativeDispatcher.obj
 0002:00001588       $unwind$Java_sun_nio_ch_Iocp_getErrorMessage 000000018000a588     Iocp.obj
 0002:00001588       $unwind$Java_sun_nio_fs_WindowsNativeDispatcher_FormatMessage 000000018000a588     WindowsNativeDispatcher.obj
 0002:000015a0       $unwind$Java_java_nio_MappedByteBuffer_force0 000000018000a5a0     MappedByteBuffer.obj
 0002:000015a0       $unwind$Java_sun_nio_fs_WindowsNativeDispatcher_initIDs 000000018000a5a0     WindowsNativeDispatcher.obj
 0002:000015b8       $unwind$Java_sun_nio_ch_Net_socket0 000000018000a5b8     Net.obj
 0002:000015c8       $unwind$Java_sun_nio_ch_Net_bind0 000000018000a5c8     Net.obj
 0002:000015dc       $unwind$Java_sun_nio_ch_Net_connect0 000000018000a5dc     Net.obj
 0002:000015fc       $unwind$Java_sun_nio_ch_Net_localInetAddress 000000018000a5fc     Net.obj
 0002:000015fc       $unwind$Java_sun_nio_ch_Net_localPort 000000018000a5fc     Net.obj
 0002:000015fc       $unwind$Java_sun_nio_ch_Net_remoteInetAddress 000000018000a5fc     Net.obj
 0002:000015fc       $unwind$Java_sun_nio_ch_Net_remotePort 000000018000a5fc     Net.obj
 0002:0000160c       $unwind$Java_sun_nio_ch_Net_getIntOption0 000000018000a60c     Net.obj
 0002:0000161c       $unwind$Java_sun_nio_ch_Net_setIntOption0 000000018000a61c     Net.obj
 0002:0000162c       $unwind$Java_sun_nio_ch_Net_poll 000000018000a62c     Net.obj
 0002:00001648       $unwind$Java_sun_nio_ch_Net_joinOrDrop4 000000018000a648     Net.obj
 0002:00001664       $unwind$Java_sun_nio_ch_Net_blockOrUnblock4 000000018000a664     Net.obj
 0002:0000167c       $unwind$Java_sun_nio_ch_Net_joinOrDrop6 000000018000a67c     Net.obj
 0002:00001690       $unwind$Java_sun_nio_ch_Net_blockOrUnblock6 000000018000a690     Net.obj
 0002:00001690       $unwind$Java_sun_nio_ch_WindowsAsynchronousFileChannelImpl_readFile 000000018000a690     WindowsAsynchronousFileChannelImpl.obj
 0002:00001690       $unwind$Java_sun_nio_ch_WindowsAsynchronousFileChannelImpl_writeFile 000000018000a690     WindowsAsynchronousFileChannelImpl.obj
 0002:00001690       $unwind$Java_sun_nio_fs_WindowsNativeDispatcher_AddAccessAllowedAceEx 000000018000a690     WindowsNativeDispatcher.obj
 0002:00001690       $unwind$Java_sun_nio_fs_WindowsNativeDispatcher_AddAccessDeniedAceEx 000000018000a690     WindowsNativeDispatcher.obj
 0002:00001690       $unwind$Java_sun_nio_fs_WindowsNativeDispatcher_CopyFileEx0 000000018000a690     WindowsNativeDispatcher.obj
 0002:00001690       $unwind$Java_sun_nio_fs_WindowsNativeDispatcher_DuplicateTokenEx 000000018000a690     WindowsNativeDispatcher.obj
 0002:00001690       $unwind$Java_sun_nio_fs_WindowsNativeDispatcher_GetFileSecurity0 000000018000a690     WindowsNativeDispatcher.obj
 0002:00001690       $unwind$Java_sun_nio_fs_WindowsNativeDispatcher_GetOverlappedResult 000000018000a690     WindowsNativeDispatcher.obj
 0002:00001690       $unwind$Java_sun_nio_fs_WindowsNativeDispatcher_GetSecurityDescriptorDacl 000000018000a690     WindowsNativeDispatcher.obj
 0002:00001690       $unwind$Java_sun_nio_fs_WindowsNativeDispatcher_GetTokenInformation 000000018000a690     WindowsNativeDispatcher.obj
 0002:00001698       $unwind$Java_sun_nio_ch_Net_getInterface4 000000018000a698     Net.obj
 0002:00001698       $unwind$Java_sun_nio_ch_Net_getInterface6 000000018000a698     Net.obj
 0002:00001698       $unwind$Java_sun_nio_ch_SocketDispatcher_preClose0 000000018000a698     SocketDispatcher.obj
 0002:00001698       $unwind$Java_sun_nio_fs_WindowsNativeDispatcher_CreateDirectory0 000000018000a698     WindowsNativeDispatcher.obj
 0002:00001698       $unwind$Java_sun_nio_fs_WindowsNativeDispatcher_ReadDirectoryChangesW 000000018000a698     WindowsNativeDispatcher.obj
 0002:000016a0       $unwind$Java_sun_nio_ch_Net_setInterface6 000000018000a6a0     Net.obj
 0002:000016a8       $unwind$setGroupSourceReqOption 000000018000a6a8     Net.obj
 0002:000016c4       $unwind$Java_sun_nio_fs_RegistryFileTypeDetector_queryStringValue 000000018000a6c4     RegistryFileTypeDetector.obj
 0002:000016dc       $unwind$Java_sun_nio_ch_ServerSocketChannelImpl_accept0 000000018000a6dc     ServerSocketChannelImpl.obj
 0002:000016f4       $unwind$Java_sun_nio_ch_SocketChannelImpl_checkConnect 000000018000a6f4     SocketChannelImpl.obj
 0002:00001710       $unwind$Java_sun_nio_ch_SocketChannelImpl_sendOutOfBandData 000000018000a710     SocketChannelImpl.obj
 0002:00001718       $unwind$Java_sun_nio_ch_SocketDispatcher_read0 000000018000a718     SocketDispatcher.obj
 0002:00001724       $unwind$Java_sun_nio_ch_SocketDispatcher_write0 000000018000a724     SocketDispatcher.obj
 0002:00001738       $unwind$Java_sun_nio_ch_SocketDispatcher_writev0 000000018000a738     SocketDispatcher.obj
 0002:00001750       $unwind$Java_sun_nio_ch_WindowsAsynchronousFileChannelImpl_lockFile 000000018000a750     WindowsAsynchronousFileChannelImpl.obj
 0002:0000175c       $unwind$Java_sun_nio_ch_WindowsAsynchronousServerSocketChannelImpl_initIDs 000000018000a75c     WindowsAsynchronousServerSocketChannelImpl.obj
 0002:0000175c       $unwind$Java_sun_nio_ch_WindowsAsynchronousSocketChannelImpl_initIDs 000000018000a75c     WindowsAsynchronousSocketChannelImpl.obj
 0002:00001774       $unwind$Java_sun_nio_ch_WindowsAsynchronousServerSocketChannelImpl_accept0 000000018000a774     WindowsAsynchronousServerSocketChannelImpl.obj
 0002:00001774       $unwind$Java_sun_nio_ch_WindowsAsynchronousSocketChannelImpl_read0 000000018000a774     WindowsAsynchronousSocketChannelImpl.obj
 0002:00001788       $unwind$Java_sun_nio_ch_WindowsAsynchronousServerSocketChannelImpl_updateAcceptContext 000000018000a788     WindowsAsynchronousServerSocketChannelImpl.obj
 0002:00001788       $unwind$Java_sun_nio_ch_WindowsAsynchronousSocketChannelImpl_updateConnectContext 000000018000a788     WindowsAsynchronousSocketChannelImpl.obj
 0002:00001790       $unwind$Java_sun_nio_ch_WindowsAsynchronousSocketChannelImpl_connect0 000000018000a790     WindowsAsynchronousSocketChannelImpl.obj
 0002:000017a4       $unwind$Java_sun_nio_ch_WindowsAsynchronousSocketChannelImpl_write0 000000018000a7a4     WindowsAsynchronousSocketChannelImpl.obj
 0002:000017b8       $unwind$Java_sun_nio_fs_WindowsNativeDispatcher_CreateFile0 000000018000a7b8     WindowsNativeDispatcher.obj
 0002:000017c4       $unwind$Java_sun_nio_fs_WindowsNativeDispatcher_DeviceIoControlGetReparsePoint 000000018000a7c4     WindowsNativeDispatcher.obj
 0002:000017c4       $unwind$Java_sun_nio_fs_WindowsNativeDispatcher_DeviceIoControlSetSparse 000000018000a7c4     WindowsNativeDispatcher.obj
 0002:000017cc       $unwind$Java_sun_nio_fs_WindowsNativeDispatcher_FindFirstFile0 000000018000a7cc     WindowsNativeDispatcher.obj
 0002:000017e8       $unwind$Java_sun_nio_fs_WindowsNativeDispatcher_FindFirstStream0 000000018000a7e8     WindowsNativeDispatcher.obj
 0002:00001804       $unwind$Java_sun_nio_fs_WindowsNativeDispatcher_FindNextStream 000000018000a804     WindowsNativeDispatcher.obj
 0002:0000181c       $unwind$Java_sun_nio_fs_WindowsNativeDispatcher_SetFileTime 000000018000a81c     WindowsNativeDispatcher.obj
 0002:00001828       $unwind$Java_sun_nio_fs_WindowsNativeDispatcher_GetVolumeInformation0 000000018000a828     WindowsNativeDispatcher.obj
 0002:00001840       $unwind$Java_sun_nio_fs_WindowsNativeDispatcher_GetDiskFreeSpaceEx0 000000018000a840     WindowsNativeDispatcher.obj
 0002:0000184c       $unwind$Java_sun_nio_fs_WindowsNativeDispatcher_GetDiskFreeSpace0 000000018000a84c     WindowsNativeDispatcher.obj
 0002:00001858       $unwind$Java_sun_nio_fs_WindowsNativeDispatcher_GetVolumePathName0 000000018000a858     WindowsNativeDispatcher.obj
 0002:00001870       $unwind$Java_sun_nio_fs_WindowsNativeDispatcher_GetAclInformation0 000000018000a870     WindowsNativeDispatcher.obj
 0002:00001884       $unwind$Java_sun_nio_fs_WindowsNativeDispatcher_LookupAccountSid0 000000018000a884     WindowsNativeDispatcher.obj
 0002:000018a0       $unwind$Java_sun_nio_fs_WindowsNativeDispatcher_LookupAccountName0 000000018000a8a0     WindowsNativeDispatcher.obj
 0002:000018b4       $unwind$Java_sun_nio_fs_WindowsNativeDispatcher_AdjustTokenPrivileges 000000018000a8b4     WindowsNativeDispatcher.obj
 0002:000018c4       $unwind$Java_sun_nio_fs_WindowsNativeDispatcher_AccessCheck 000000018000a8c4     WindowsNativeDispatcher.obj
 0002:000018dc       $unwind$Java_sun_nio_fs_WindowsNativeDispatcher_GetFinalPathNameByHandle 000000018000a8dc     WindowsNativeDispatcher.obj
 0002:000018dc       $unwind$Java_sun_nio_fs_WindowsNativeDispatcher_GetFullPathName0 000000018000a8dc     WindowsNativeDispatcher.obj
 0002:000018fc       $unwind$Java_sun_nio_ch_WindowsSelectorImpl_resetWakeupSocket0 000000018000a8fc     WindowsSelectorImpl.obj
 0002:00001914       $unwind$Java_sun_nio_ch_WindowsSelectorImpl_discardUrgentData 000000018000a914     WindowsSelectorImpl.obj
 0002:00001928       $unwind$Java_sun_nio_ch_WindowsSelectorImpl_00024SubSelector_poll0 000000018000a928     WindowsSelectorImpl.obj
 0002:00001950       $unwind$__GSHandlerCheckCommon 000000018000a950     MSVCRT:gshandler.obj
 0002:00001958       $xdatasym                  000000018000a958     MSVCRT:amdsecgs.obj
 0002:00001960       $xdatasym                  000000018000a960     MSVCRT:chkstk.obj
 0002:00001968       $unwind$?dllmain_crt_process_attach@@YAHQEAUHINSTANCE__@@QEAX@Z 000000018000a968     MSVCRT:dll_dllmain.obj
 0002:000019a4       $unwind$?fin$0@?0??dllmain_crt_process_attach@@YAHQEAUHINSTANCE__@@QEAX@Z@4HA 000000018000a9a4     MSVCRT:dll_dllmain.obj
 0002:000019a4       $unwind$?fin$0@?0??dllmain_crt_process_detach@@YAH_N@Z@4HA 000000018000a9a4     MSVCRT:dll_dllmain.obj
 0002:000019a4       $unwind$?fin$1@?0??dllmain_crt_process_detach@@YAH_N@Z@4HA 000000018000a9a4     MSVCRT:dll_dllmain.obj
 0002:000019ac       $unwind$?dllmain_crt_process_detach@@YAH_N@Z 000000018000a9ac     MSVCRT:dll_dllmain.obj
 0002:00001a00       $unwind$?dllmain_dispatch@@YAHQEAUHINSTANCE__@@KQEAX@Z 000000018000aa00     MSVCRT:dll_dllmain.obj
 0002:00001a28       $unwind$?filt$0@?0??dllmain_dispatch@@YAHQEAUHINSTANCE__@@KQEAX@Z@4HA 000000018000aa28     MSVCRT:dll_dllmain.obj
 0002:00001a30       $unwind$__report_gsfailure 000000018000aa30     MSVCRT:gs_report.obj
 0002:00001a38       $unwind$capture_previous_context 000000018000aa38     MSVCRT:gs_report.obj
 0002:00001a44       $unwind$__security_init_cookie 000000018000aa44     MSVCRT:gs_support.obj
 0002:00001a50       $unwind$__scrt_is_nonwritable_in_current_image 000000018000aa50     MSVCRT:utility.obj
 0002:00001a70       $unwind$__scrt_is_nonwritable_in_current_image$filt$0 000000018000aa70     MSVCRT:utility.obj
 0002:00001a78       $unwind$__scrt_dllmain_exception_filter 000000018000aa78     MSVCRT:utility.obj
 0002:00001a8c       $unwind$__scrt_fastfail    000000018000aa8c     MSVCRT:utility_desktop.obj
 0002:00001a9c       $unwind$__isa_available_init 000000018000aa9c     MSVCRT:cpu_disp.obj
 0002:00001ab0       $xdatasym                  000000018000aab0     MSVCRT:guard_dispatch.obj
 0002:00001ab8       $xdatasym                  000000018000aab8     MSVCRT:guard_xfg_dispatch.obj
 0002:00001ac0       .edata                     000000018000aac0     nio.exp
 0002:00001ae8       rgpv                       000000018000aae8     nio.exp
 0002:00001dac       rgszName                   000000018000adac     nio.exp
 0002:00002070       rgwOrd                     000000018000b070     nio.exp
 0002:000021d2       szName                     000000018000b1d2     nio.exp
 0002:000021da       $N00001                    000000018000b1da     nio.exp
 0002:000021e5       $N00002                    000000018000b1e5     nio.exp
 0002:0000220b       $N00003                    000000018000b20b     nio.exp
 0002:00002234       $N00004                    000000018000b234     nio.exp
 0002:00002259       $N00005                    000000018000b259     nio.exp
 0002:00002289       $N00006                    000000018000b289     nio.exp
 0002:000022b5       $N00007                    000000018000b2b5     nio.exp
 0002:000022e2       $N00008                    000000018000b2e2     nio.exp
 0002:0000230c       $N00009                    000000018000b30c     nio.exp
 0002:00002335       $N00010                    000000018000b335     nio.exp
 0002:0000235f       $N00011                    000000018000b35f     nio.exp
 0002:00002389       $N00012                    000000018000b389     nio.exp
 0002:000023b4       $N00013                    000000018000b3b4     nio.exp
 0002:000023dc       $N00014                    000000018000b3dc     nio.exp
 0002:00002401       $N00015                    000000018000b401     nio.exp
 0002:0000242d       $N00016                    000000018000b42d     nio.exp
 0002:00002454       $N00017                    000000018000b454     nio.exp
 0002:0000247e       $N00018                    000000018000b47e     nio.exp
 0002:000024b1       $N00019                    000000018000b4b1     nio.exp
 0002:000024db       $N00020                    000000018000b4db     nio.exp
 0002:00002504       $N00021                    000000018000b504     nio.exp
 0002:0000252e       $N00022                    000000018000b52e     nio.exp
 0002:00002559       $N00023                    000000018000b559     nio.exp
 0002:00002582       $N00024                    000000018000b582     nio.exp
 0002:000025ac       $N00025                    000000018000b5ac     nio.exp
 0002:000025d8       $N00026                    000000018000b5d8     nio.exp
 0002:00002601       $N00027                    000000018000b601     nio.exp
 0002:0000262f       $N00028                    000000018000b62f     nio.exp
 0002:00002658       $N00029                    000000018000b658     nio.exp
 0002:00002685       $N00030                    000000018000b685     nio.exp
 0002:000026af       $N00031                    000000018000b6af     nio.exp
 0002:000026da       $N00032                    000000018000b6da     nio.exp
 0002:000026f7       $N00033                    000000018000b6f7     nio.exp
 0002:00002717       $N00034                    000000018000b717     nio.exp
 0002:00002740       $N00035                    000000018000b740     nio.exp
 0002:0000275d       $N00036                    000000018000b75d     nio.exp
 0002:0000277a       $N00037                    000000018000b77a     nio.exp
 0002:00002799       $N00038                    000000018000b799     nio.exp
 0002:000027b7       $N00039                    000000018000b7b7     nio.exp
 0002:000027da       $N00040                    000000018000b7da     nio.exp
 0002:000027fa       $N00041                    000000018000b7fa     nio.exp
 0002:00002816       $N00042                    000000018000b816     nio.exp
 0002:00002842       $N00043                    000000018000b842     nio.exp
 0002:00002867       $N00044                    000000018000b867     nio.exp
 0002:00002896       $N00045                    000000018000b896     nio.exp
 0002:000028b3       $N00046                    000000018000b8b3     nio.exp
 0002:000028e3       $N00047                    000000018000b8e3     nio.exp
 0002:000028fd       $N00048                    000000018000b8fd     nio.exp
 0002:00002921       $N00049                    000000018000b921     nio.exp
 0002:00002945       $N00050                    000000018000b945     nio.exp
 0002:00002975       $N00051                    000000018000b975     nio.exp
 0002:000029a0       $N00052                    000000018000b9a0     nio.exp
 0002:000029bd       $N00053                    000000018000b9bd     nio.exp
 0002:000029df       $N00054                    000000018000b9df     nio.exp
 0002:00002a01       $N00055                    000000018000ba01     nio.exp
 0002:00002a23       $N00056                    000000018000ba23     nio.exp
 0002:00002a3f       $N00057                    000000018000ba3f     nio.exp
 0002:00002a6c       $N00058                    000000018000ba6c     nio.exp
 0002:00002a91       $N00059                    000000018000ba91     nio.exp
 0002:00002abb       $N00060                    000000018000babb     nio.exp
 0002:00002adb       $N00061                    000000018000badb     nio.exp
 0002:00002afb       $N00062                    000000018000bafb     nio.exp
 0002:00002b16       $N00063                    000000018000bb16     nio.exp
 0002:00002b3b       $N00064                    000000018000bb3b     nio.exp
 0002:00002b59       $N00065                    000000018000bb59     nio.exp
 0002:00002b72       $N00066                    000000018000bb72     nio.exp
 0002:00002b94       $N00067                    000000018000bb94     nio.exp
 0002:00002bb5       $N00068                    000000018000bbb5     nio.exp
 0002:00002bd6       $N00069                    000000018000bbd6     nio.exp
 0002:00002bf6       $N00070                    000000018000bbf6     nio.exp
 0002:00002c18       $N00071                    000000018000bc18     nio.exp
 0002:00002c39       $N00072                    000000018000bc39     nio.exp
 0002:00002c5f       $N00073                    000000018000bc5f     nio.exp
 0002:00002c7e       $N00074                    000000018000bc7e     nio.exp
 0002:00002ca0       $N00075                    000000018000bca0     nio.exp
 0002:00002cc2       $N00076                    000000018000bcc2     nio.exp
 0002:00002ce4       $N00077                    000000018000bce4     nio.exp
 0002:00002d01       $N00078                    000000018000bd01     nio.exp
 0002:00002d1d       $N00079                    000000018000bd1d     nio.exp
 0002:00002d4d       $N00080                    000000018000bd4d     nio.exp
 0002:00002d7d       $N00081                    000000018000bd7d     nio.exp
 0002:00002dac       $N00082                    000000018000bdac     nio.exp
 0002:00002ddb       $N00083                    000000018000bddb     nio.exp
 0002:00002e05       $N00084                    000000018000be05     nio.exp
 0002:00002e39       $N00085                    000000018000be39     nio.exp
 0002:00002e61       $N00086                    000000018000be61     nio.exp
 0002:00002e8c       $N00087                    000000018000be8c     nio.exp
 0002:00002eb3       $N00088                    000000018000beb3     nio.exp
 0002:00002edb       $N00089                    000000018000bedb     nio.exp
 0002:00002f03       $N00090                    000000018000bf03     nio.exp
 0002:00002f2c       $N00091                    000000018000bf2c     nio.exp
 0002:00002f68       $N00092                    000000018000bf68     nio.exp
 0002:00002fa4       $N00093                    000000018000bfa4     nio.exp
 0002:00002fe1       $N00094                    000000018000bfe1     nio.exp
 0002:00003024       $N00095                    000000018000c024     nio.exp
 0002:0000306c       $N00096                    000000018000c06c     nio.exp
 0002:000030af       $N00097                    000000018000c0af     nio.exp
 0002:000030fe       $N00098                    000000018000c0fe     nio.exp
 0002:00003140       $N00099                    000000018000c140     nio.exp
 0002:0000317e       $N00100                    000000018000c17e     nio.exp
 0002:000031bb       $N00101                    000000018000c1bb     nio.exp
 0002:000031f6       $N00102                    000000018000c1f6     nio.exp
 0002:00003235       $N00103                    000000018000c235     nio.exp
 0002:0000327f       $N00104                    000000018000c27f     nio.exp
 0002:000032bb       $N00105                    000000018000c2bb     nio.exp
 0002:000032f6       $N00106                    000000018000c2f6     nio.exp
 0002:0000332c       $N00107                    000000018000c32c     nio.exp
 0002:00003363       $N00108                    000000018000c363     nio.exp
 0002:00003398       $N00109                    000000018000c398     nio.exp
 0002:000033d2       $N00110                    000000018000c3d2     nio.exp
 0002:00003406       $N00111                    000000018000c406     nio.exp
 0002:00003444       $N00112                    000000018000c444     nio.exp
 0002:00003481       $N00113                    000000018000c481     nio.exp
 0002:000034bf       $N00114                    000000018000c4bf     nio.exp
 0002:000034f0       $N00115                    000000018000c4f0     nio.exp
 0002:00003524       $N00116                    000000018000c524     nio.exp
 0002:00003562       $N00117                    000000018000c562     nio.exp
 0002:000035a1       $N00118                    000000018000c5a1     nio.exp
 0002:000035d5       $N00119                    000000018000c5d5     nio.exp
 0002:0000360e       $N00120                    000000018000c60e     nio.exp
 0002:00003642       $N00121                    000000018000c642     nio.exp
 0002:00003676       $N00122                    000000018000c676     nio.exp
 0002:000036ae       $N00123                    000000018000c6ae     nio.exp
 0002:000036ed       $N00124                    000000018000c6ed     nio.exp
 0002:00003729       $N00125                    000000018000c729     nio.exp
 0002:0000375d       $N00126                    000000018000c75d     nio.exp
 0002:000037a4       $N00127                    000000018000c7a4     nio.exp
 0002:000037e5       $N00128                    000000018000c7e5     nio.exp
 0002:0000381e       $N00129                    000000018000c81e     nio.exp
 0002:00003850       $N00130                    000000018000c850     nio.exp
 0002:00003887       $N00131                    000000018000c887     nio.exp
 0002:000038be       $N00132                    000000018000c8be     nio.exp
 0002:000038f7       $N00133                    000000018000c8f7     nio.exp
 0002:0000392c       $N00134                    000000018000c92c     nio.exp
 0002:00003963       $N00135                    000000018000c963     nio.exp
 0002:00003999       $N00136                    000000018000c999     nio.exp
 0002:000039c8       $N00137                    000000018000c9c8     nio.exp
 0002:00003a03       $N00138                    000000018000ca03     nio.exp
 0002:00003a3d       $N00139                    000000018000ca3d     nio.exp
 0002:00003a76       $N00140                    000000018000ca76     nio.exp
 0002:00003ab0       $N00141                    000000018000cab0     nio.exp
 0002:00003aec       $N00142                    000000018000caec     nio.exp
 0002:00003b22       $N00143                    000000018000cb22     nio.exp
 0002:00003b5d       $N00144                    000000018000cb5d     nio.exp
 0002:00003b9a       $N00145                    000000018000cb9a     nio.exp
 0002:00003bdd       $N00146                    000000018000cbdd     nio.exp
 0002:00003c16       $N00147                    000000018000cc16     nio.exp
 0002:00003c57       $N00148                    000000018000cc57     nio.exp
 0002:00003c90       $N00149                    000000018000cc90     nio.exp
 0002:00003cc5       $N00150                    000000018000ccc5     nio.exp
 0002:00003cfe       $N00151                    000000018000ccfe     nio.exp
 0002:00003d3a       $N00152                    000000018000cd3a     nio.exp
 0002:00003d7d       $N00153                    000000018000cd7d     nio.exp
 0002:00003dbf       $N00154                    000000018000cdbf     nio.exp
 0002:00003e02       $N00155                    000000018000ce02     nio.exp
 0002:00003e3e       $N00156                    000000018000ce3e     nio.exp
 0002:00003e7c       $N00157                    000000018000ce7c     nio.exp
 0002:00003eb7       $N00158                    000000018000ceb7     nio.exp
 0002:00003eed       $N00159                    000000018000ceed     nio.exp
 0002:00003f32       $N00160                    000000018000cf32     nio.exp
 0002:00003f64       $N00161                    000000018000cf64     nio.exp
 0002:00003f9f       $N00162                    000000018000cf9f     nio.exp
 0002:00003fd9       $N00163                    000000018000cfd9     nio.exp
 0002:00004017       $N00164                    000000018000d017     nio.exp
 0002:0000404b       $N00165                    000000018000d04b     nio.exp
 0002:00004084       $N00166                    000000018000d084     nio.exp
 0002:000040bc       $N00167                    000000018000d0bc     nio.exp
 0002:000040ff       $N00168                    000000018000d0ff     nio.exp
 0002:0000413d       $N00169                    000000018000d13d     nio.exp
 0002:00004176       $N00170                    000000018000d176     nio.exp
 0002:000041ab       $N00171                    000000018000d1ab     nio.exp
 0002:000041e6       $N00172                    000000018000d1e6     nio.exp
 0002:0000421f       $N00173                    000000018000d21f     nio.exp
 0002:00004253       $N00174                    000000018000d253     nio.exp
 0002:00004295       $N00175                    000000018000d295     nio.exp
 0002:000042d8       $N00176                    000000018000d2d8     nio.exp
 0002:0000430f       $N00177                    000000018000d30f     nio.exp
 0002:000049c2       .idata$6                   000000018000d9c2     ws2_32:WS2_32.dll
 0002:00004a94       .idata$6                   000000018000da94     java:java.dll
 0002:00004bba       .idata$6                   000000018000dbba     net:net.dll
 0002:00004e2e       .idata$6                   000000018000de2e     advapi32:ADVAPI32.dll
 0002:00004e4c       .idata$6                   000000018000de4c     Mswsock:MSWSOCK.dll
 0002:000053f2       .idata$6                   000000018000e3f2     kernel32:KERNEL32.dll
 0002:00005442       .idata$6                   000000018000e442     vcruntime:VCRUNTIME140.dll
 0002:00005532       .idata$6                   000000018000e532     ucrt:api-ms-win-crt-heap-l1-1-0.dll
 0002:00005552       .idata$6                   000000018000e552     ucrt:api-ms-win-crt-stdio-l1-1-0.dll
 0002:00005572       .idata$6                   000000018000e572     ucrt:api-ms-win-crt-string-l1-1-0.dll
 0002:00005594       .idata$6                   000000018000e594     ucrt:api-ms-win-crt-runtime-l1-1-0.dll
 0003:00000000       ?loopback_available@?6??Java_sun_nio_ch_Net_socket0@@9@9 000000018000f000     Net.obj
 0003:00000050       dci_senderID               000000018000f050     DatagramChannelImpl.obj
 0003:00000058       dci_senderAddrID           000000018000f058     DatagramChannelImpl.obj
 0003:00000060       dci_senderPortID           000000018000f060     DatagramChannelImpl.obj
 0003:00000068       isa_class                  000000018000f068     DatagramChannelImpl.obj
 0003:00000070       isa_ctorID                 000000018000f070     DatagramChannelImpl.obj
 0003:00000078       chan_fd                    000000018000f078     FileChannelImpl.obj
 0003:00000080       key_volumeSN               000000018000f080     FileKey.obj
 0003:00000088       key_indexHigh              000000018000f088     FileKey.obj
 0003:00000090       key_indexLow               000000018000f090     FileKey.obj
 0003:00000098       handle_fdID                000000018000f098     IOUtil.obj
 0003:000000a0       fd_fdID                    000000018000f0a0     IOUtil.obj
 0003:000000a8       completionStatus_error     000000018000f0a8     Iocp.obj
 0003:000000b0       completionStatus_bytesTransferred 000000018000f0b0     Iocp.obj
 0003:000000b8       completionStatus_completionKey 000000018000f0b8     Iocp.obj
 0003:000000c0       completionStatus_overlapped 000000018000f0c0     Iocp.obj
 0003:000000c8       ?handle_fdID@?3??Java_java_nio_MappedByteBuffer_force0@@9@9 000000018000f0c8     MappedByteBuffer.obj
 0003:000000d0       fd_fdID                    000000018000f0d0     ServerSocketChannelImpl.obj
 0003:000000d8       isa_class                  000000018000f0d8     ServerSocketChannelImpl.obj
 0003:000000e0       isa_ctorID                 000000018000f0e0     ServerSocketChannelImpl.obj
 0003:000000e8       ia_addrID                  000000018000f0e8     SocketChannelImpl.obj
 0003:000000f0       AcceptEx_func              000000018000f0f0     WindowsAsynchronousServerSocketChannelImpl.obj
 0003:000000f8       ConnectEx_func             000000018000f0f8     WindowsAsynchronousSocketChannelImpl.obj
 0003:00000100       findFirst_handle           000000018000f100     WindowsNativeDispatcher.obj
 0003:00000108       findFirst_name             000000018000f108     WindowsNativeDispatcher.obj
 0003:00000110       findFirst_attributes       000000018000f110     WindowsNativeDispatcher.obj
 0003:00000118       findStream_handle          000000018000f118     WindowsNativeDispatcher.obj
 0003:00000120       findStream_name            000000018000f120     WindowsNativeDispatcher.obj
 0003:00000128       volumeInfo_fsName          000000018000f128     WindowsNativeDispatcher.obj
 0003:00000130       volumeInfo_volName         000000018000f130     WindowsNativeDispatcher.obj
 0003:00000138       volumeInfo_volSN           000000018000f138     WindowsNativeDispatcher.obj
 0003:00000140       volumeInfo_flags           000000018000f140     WindowsNativeDispatcher.obj
 0003:00000148       diskSpace_bytesAvailable   000000018000f148     WindowsNativeDispatcher.obj
 0003:00000150       diskSpace_totalBytes       000000018000f150     WindowsNativeDispatcher.obj
 0003:00000158       diskSpace_totalFree        000000018000f158     WindowsNativeDispatcher.obj
 0003:00000160       diskSpace_bytesPerSector   000000018000f160     WindowsNativeDispatcher.obj
 0003:00000168       account_domain             000000018000f168     WindowsNativeDispatcher.obj
 0003:00000170       account_name               000000018000f170     WindowsNativeDispatcher.obj
 0003:00000178       account_use                000000018000f178     WindowsNativeDispatcher.obj
 0003:00000180       aclInfo_aceCount           000000018000f180     WindowsNativeDispatcher.obj
 0003:00000188       completionStatus_error     000000018000f188     WindowsNativeDispatcher.obj
 0003:00000190       completionStatus_bytesTransferred 000000018000f190     WindowsNativeDispatcher.obj
 0003:00000198       completionStatus_completionKey 000000018000f198     WindowsNativeDispatcher.obj
 0003:000001a0       ?zerotime@?1??Java_sun_nio_ch_WindowsSelectorImpl_00024SubSelector_poll0@@9@9 000000018000f1a0     WindowsSelectorImpl.obj
 0003:000001a8       ?__proc_attached@@3HA      000000018000f1a8     MSVCRT:dll_dllmain.obj
 0003:000001b0       GS_ExceptionRecord         000000018000f1b0     MSVCRT:gs_report.obj
 0003:00000250       GS_ContextRecord           000000018000f250     MSVCRT:gs_report.obj
 0003:00000750       ?is_initialized_as_dll@@3_NA 000000018000f750     MSVCRT:utility.obj
 0003:00000751       ?module_local_atexit_table_initialized@@3_NA 000000018000f751     MSVCRT:utility.obj
 0003:00000758       ?module_local_atexit_table@@3U_onexit_table_t@@A 000000018000f758     MSVCRT:utility.obj
 0003:00000770       ?module_local_at_quick_exit_table@@3U_onexit_table_t@@A 000000018000f770     MSVCRT:utility.obj
 0005:00000060       $R000000                   0000000180011060     nio.dll.res
